S02000006F70656E626C745F6F6C696D65785F73746D3332703430352E7372656302
S3150800000000000220BD0A00088D0A00088F0A0008B1
S31508000010910A0008930A0008950A000800000000E3
S31508000020000000000000000000000000970A000819
S31508000030990A0008000000009B0A00089D0A0008AB
S315080000400D0B00080D0B00080D0B00080D0B000822
S315080000500D0B00080D0B00080D0B00080D0B000812
S315080000600D0B00080D0B00080D0B00080D0B000802
S315080000700D0B00080D0B00080D0B00080D0B0008F2
S315080000800D0B00080D0B00080D0B00080D0B0008E2
S315080000900D0B00080D0B00080D0B00080D0B0008D2
S315080000A00D0B00080D0B00080D0B00080D0B0008C2
S315080000B00D0B00080D0B00080D0B00080D0B0008B2
S315080000C00D0B00080D0B00080D0B00080D0B0008A2
S315080000D00D0B00080D0B00080D0B00080D0B000892
S315080000E00D0B00080D0B00080D0B00080D0B000882
S315080000F00D0B00080D0B00080D0B00080D0B000872
S315080001000D0B00080D0B00080D0B00080D0B000861
S315080001100D0B00080D0B00080D0B00080D0B000851
S315080001200D0B00080D0B00080D0B00080D0B000841
S315080001300D0B000800000000000000000D0B000871
S315080001400D0B00080D0B00080D0B00080D0B000821
S315080001500D0B00080D0B00080D0B00080D0B000811
S315080001600D0B00080D0B00080D0B00080D0B000801
S315080001700D0B00080D0B0008000000000000000031
S30D080001800D0B00080D0B000829
S3150800018810B5054C237833B9044B13B10448AFF3BB
S3150800019800800123237010BD7802002000000000AB
S315080001A88C73000808B5034B1BB103490348AFF322
S315080001B8008008BD000000007C0200208C7300083F
S315080001C853B94AB9002908BF00281CBF4FF0FF31A8
S315080001D84FF0FF3000F072B9ADF1080C6DE904CEA6
S315080001E800F006F8DDF804E0DDE9022304B07047FC
S315080001F82DE9F047089E04468846002B4BD18A42CB
S31508000208154667D9B2FA82F24AB1C2F1200701FA4D
S3150800021802F320FA07F7954047EA030894404FEA9D
S31508000228154E230CB8FBFEF71FFA85FC0EFB17883C
S3150800023843EA084307FB0CF1994209D9EB1807F179
S31508000248FF3080F01B81994240F21881023F2B4407
S315080002585B1AA4B2B3FBFEF00EFB103344EA034460
S3150800026800FB0CFCA44509D92C1900F1FF3380F0D2
S315080002780781A44540F2048102382C4440EA074025
S31508000288A4EB0C0400271EB1D4400023C6E900439A
S315080002983946BDE8F0878B4209D9002E00F0EB8075
S315080002A80027C6E9000138463946BDE8F087B3FA9B
S315080002B883F7002F47D18B4202D3824200F2FA8095
S315080002C8841A61EB030301209846002EE0D0C6E99C
S315080002D80048DDE702B9FFDEB2FA82F2002A40F0EA
S315080002E88F80491B4FEA154E1FFA85F80127B1FB7F
S315080002F8FEFC230C0EFB1C1143EA014308FB0CF118
S31508000308994207D9EB180CF1FF3002D2994200F24C
S31508000318CD808446591AA3B2B1FBFEF00EFB101421
S3150800032843EA044408FB00F8A04507D92C1900F14C
S31508000338FF3302D2A04500F2B6801846A4EB08049B
S3150800034840EA0C409FE7C7F1200CBB4022FA0CFE96
S315080003584EEA030E01FA07F420FA0CF521FA0CF313
S315080003684FEA1E482543B3FBF8F92C0C08FB19334A
S315080003781FFA8EFA44EA034309FB0AF49C4202FA76
S3150800038807F200FA07F10BD91EEB030309F1FF3050
S3150800039880F087809C4240F28480A9F10209734460
S315080003A81B1BADB2B3FBF8F008FB103345EA034450
S315080003B800FB0AFAA24508D91EEB040400F1FF332C
S315080003C86BD2A24569D90238744440EA0940A0FBB1
S315080003D80289A4EB0A044C45C2464B4654D351D06D
S315080003E8002E69D0B1EB0A0564EB030404FA0CFC89
S315080003F8FD40FC404CEA0505C6E90054002747E7D6
S31508000408C2F1200320FA03F7954001FA02F021FA0F
S3150800041803F34FEA154E3843010CB3FBFEF71FFAF0
S3150800042885F80EFB173341EA034107FB08F38B42AD
S3150800043804FA02F407D9691807F1FF3C2FD28B4250
S315080004482DD9023F2944CB1A81B2B3FBFEF00EFB25
S31508000458103341EA034100FB08F38B4207D96918B0
S3150800046800F1FF3C17D28B4215D902382944C91A1C
S3150800047840EA07473BE73746304609E70746E7E6CF
S315080004881846FBE64145ABD2B8EB020A69EB0E0201
S3150800049801381346A4E76046E9E7184695E767462C
S315080004A8D1E781467CE702382C4447E7ACF1020CD1
S315080004B82B442FE7384608E73746E9E6704700BF72
S315080004C804F074BA04F083BA08B5054B1B69DB0750
S315080004D803D400F0F1F8012008BD0020FCE700BFAE
S315080004E800000240642000F0BDB800F0C1B8000062
S315080004F870B5134D2B7888B00646B3B9114A124819
S31508000508116B41F004011163126B069302F00402A1
S3150800051801920124019A02A94FF40062CDE9022446
S31508000528CDE9043401F084FE2C70012E064B0CBF6D
S315080005384FF000624FF400629A6108B070BD00BFC0
S3150800054894020020003802400008024070477047AD
S3150800055800B5C7B000214FF48C72684606F0FCFE59
S315080005686946084806F07AFB50B9009828B19DF8FC
S31508000578080080F01000C0F3001047B05DF804FBCF
S315080005880020FAE7B173000800487047B1730008FD
S3150800059810B5074C074900230A22204684F8283252
S315080005A806F03AF810B9012384F8283210BD00BFBE
S315080005B898020020A473000838B50C4890F8283229
S315080005C8012B01D106F0A4FA03F0F8FF084C00F154
S315080005D8640523685B0603D403F0F0FFA842F8D93C
S315080005E80448BDE8384006F063BB00BF98020020FF
S315080005F800440040B1730008034890F82832012BDC
S3150800060801D106F085BA70479802002070B5134DD7
S3150800061895F82832012B04460AD1294606F0C3FB69
S31508000628002805DA0023284685F8283206F070FAE5
S315080006380B4D013C14F8013F03B970BD6B6003F01C
S31508000648BDFF00F10A062B681B06F3D404F04DFA21
S3150800065803F0B4FFB042F6D9ECE700BF98020020D1
S3150800066800440040014B1880704700BFC4040020AE
S3150800067810B50D4C03F0A2FF226890420ED30B4B1F
S315080006880B4A197859B9012119704FF080539361AB
S3150800069803F094FF074B1B881844206010BD0021FF
S315080006A819704FF48053F2E7C8040020C6040020E6
S315080006B800080240C4040020024B4FF480529A6195
S315080006C8704700BF00080240054B1A6B02431A63BD
S315080006D81B6B82B018400190019B02B0704700BF9F
S315080006E80038024008B52A4B1A6822F00F0242F071
S315080006F805021A601A6802F00F02052AFAD1254A75
S31508000708136843F480431360234B1A6842F4803213
S315080007181A601A689103FCD55A6820491140204A7C
S315080007280A435A605A681F4922F440325A605A687E
S3150800073811401D4A0A435A601A6842F080721A60C4
S31508000748154B1A689201FCD59A6822F0F0029A604D
S315080007589A6822F4E05242F4A0529A609A6822F4FF
S31508000768604242F400429A609A6822F0030242F014
S3150800077802029A60084A936803F00C03082BFAD118
S315080007880A4802F043FC0020BDE8084000F0D2B948
S31508000798003C024000700040003802400080BFFF5D
S315080007A8085440000080BFF008544007007A030A3E
S315080007B880B58EB000F0E2F9FFF794FF1822002101
S315080007C807A806F0C9FD8020FFF77EFF0120FFF77E
S315080007D87BFFDFF8EC90DFF8EC800220FFF774FF68
S315080007E84FF4805604200024FFF76EFF0125C9F848
S315080007F8186007A9C8F818602E480B94CDE907545D
S31508000808022701F015FD07A94846CDE90765CDE990
S3150800081809740B9401F00CFD07A94046CDE9076554
S31508000828CDE909440B9401F003FD1C2221460DEB82
S31508000838020006F091FD2146182201A806F08CFD53
S315080008481D4B1A6C42F400321A641B6C03F400330D
S3150800085828460093009BFFF737FF0323CDE90334A7
S315080008680C25072301A9134805940693CDE90157D2
S3150800087801F0DEFC4FF4E133CDE90734CDE909444C
S31508000888CDE90B540D940D4C07A9204601F058FEE6
S31508000898236923F490432361636923F02A03636178
S315080008A8E36843F40053E360FFF70AFEFFF70AFE1E
S315080008B8FCE700BF00000240003802400044004040
S315080008C8000402400008024082B00C4B0021009147
S315080008D85A6C42F480425A645A6C02F48042009276
S315080008E8009A01911A6C42F080521A641B6C03F044
S315080008F880530193019B02B0704700BF003802403D
S3150800090810B5044688B01422002103A806F024FD71
S315080009182268144B9A4223D103F5EA330021019140
S315080009281A6C114842F000721A641A6C02F00072C6
S315080009380192019A02911A6B42F002021A631B6B22
S3150800094803F002030293029B4FF440720223032129
S31508000958CDE903230923CDE9061303A900F054FDBD
S3150800096808B010BD006400400004024030B50446D3
S3150800097889B01422002103A806F0EEFC2368B3F117
S31508000988A04F26D1144C154800250195236B43F032
S3150800099801032363236B03F001030193019B4FF4BF
S315080009A8C0520223CDE9032303210A23CDE90613FE
S315080009B803A900F029FD636B43F08003636302957E
S315080009C8636C43F480436364636C03F48043029363
S315080009D8029B09B030BD00BF003802400000024043
S315080009E80368B3F1A04F09D1054A0648536B23F0AB
S315080009F8800353634FF4C05100F0E6BD704700BF4B
S31508000A08003802400000024010B5194C01F0AEFC4F
S31508000A18636B184823F08003636301F0A7FB164845
S31508000A2801F0A4FB154801F0A1FB236C144A23F036
S31508000A3800732364D36823F40053D360236C23F428
S31508000A4800332364236B23F004032363236B23F007
S31508000A5802032363236B23F001032363236C23F028
S31508000A6880532364636C23F48043636410BD00BF1A
S31508000A780038024000080240000402400000024014
S31508000A88004400407047FEE7FEE7FEE7FEE77047CA
S31508000A987047704700F08CB8054BD3F8882042F4A5
S31508000AA87002C3F888204FF000629A60704700BF4A
S31508000AB800ED00E0DFF834D0002103E00C4B5B586A
S31508000AC8435004310B480C4B42189A42F6D30B4A4A
S31508000AD802E0002342F8043B094B9A42F9D3FFF790
S31508000AE8DBFF06F0F5FBFFF763FE70470000022000
S31508000AF8D47C000800000020780200207802002034
S31508000B08BC1C0020FEE7000010B5094B4FF0FF3269
S31508000B1800241A621C625A625C621A611C615A6174
S31508000B285C619A619C61FFF76FFF204610BD00BFA4
S31508000B380038024038B50E4A0E4B054618784FF469
S31508000B487A73B3FBF0F31068B0FBF3F000F094FA8D
S31508000B58044658B90F2D09D8024629464FF0FF30E2
S31508000B6800F056FA044B20461D6038BD0120FCE704
S31508000B7800000020040000200800002008B50B4BE0
S31508000B881A6842F400721A601A6842F480621A6097
S31508000B981A6842F480721A60032000F027FA0020C7
S31508000BA8FFF7C8FFFFF790FE002008BD003C02408B
S31508000BB8034A044B11681B780B441360704700BF3F
S31508000BC8581A00200400002038B5044603F0FEFC35
S31508000BD8631C1CBF054B1B78054618BFE41803F0B1
S31508000BE8F5FC401BA042FAD338BD00BF040000201C
S31508000BF838B5044600286ED090F820300BB9FFF7B0
S31508000C087FFE2268136823F00203136003F0DEFCF4
S31508000C18054623685A68910751D41A6842F00102B2
S31508000C281A6003F0D3FC054623685A68D20754D5D8
S31508000C38227E012A1A680CBF42F0800222F080023E
S31508000C481A60627E012A1A680CBF42F0400222F036
S31508000C5840021A60A27E012A1A680CBF42F02002D6
S31508000C6822F020021A60E27E012A1A680CBF22F0D6
S31508000C78100242F010021A60227F012A1A680CBF75
S31508000C8842F0080222F008021A60627F012A1A68EE
S31508000C980CBF42F0040222F004021A60D4E90221C9
S31508000CA80A4321690A4361690A43616801390A43A3
S31508000CB8DA6100200123606284F8203038BD03F029
S31508000CC885FC401B0A28A4D9636A43F40033636287
S31508000CD8052384F820300120F0E703F077FC401B51
S31508000CE80A28A1D9F0E7000090F82030013B012B2B
S31508000CF830B574D83D4BD3F8002242F00102C3F848
S31508000D080022D3F8002222F47C52C3F80022D3F832
S31508000D180022486A42EA0022C3F800224869D3F842
S31508000D281C5200F01F0201249440E2431540C3F800
S31508000D381C52CD69002D35D1D3F80C521540C3F88D
S31508000D480C52CB688D8845EA0345C30003F18043F6
S31508000D5803F5C8430888C3F840528D6840EA054039
S31508000D68C3F844028869214B88BBD3F804021040AB
S31508000D78C3F80402086970BBD3F814020240C3F822
S31508000D8814220B6A012B194B02BFD3F81C221443F1
S31508000D98C3F81C42D3F8002222F00102C3F8002245
S31508000DA8002030BD012DDDD1D3F80C522543C3F8F8
S31508000DB80C520B688D8845EA0345C30003F1804346
S31508000DC803F5C8438889C3F840528D68C6E7D3F83F
S31508000DD804022043CCE7D3F814222243CFE7436A18
S31508000DE843F4802343620120DBE700BF0064004028
S31508000DF838B590F82030012B04461FD10268022323
S31508000E0880F82030136823F00103136003F0DEFB33
S31508000E1805462368586810F0010001D1606238BD9C
S31508000E2803F0D4FB401B0A28F3D9636A43F400335A
S31508000E386362052384F820300120F0E7436A43F407
S31508000E4800234362F8E7F0B590F820500668013D9C
S31508000E58012DB46840D814F0E05F39D0C4F30164B2
S31508000E68032C4FF0010505D1436A43F40003436296
S31508000E78012027E0A5401D60D1E9020704F11803FF
S31508000E8808BB086847EA40501B012401F05033198B
S31508000E980869097DC3F88401012902BFD3F88411BA
S31508000EA841F48071C3F8841134445168C4F88C112C
S31508000EB81268C4F88821D3F8802142F00102C3F8E1
S31508000EC880210020F0BD4D68384340EAC500DBE7BD
S31508000ED8436A43F40013CAE7436A43F48023C6E720
S31508000EE890F82030013B012B08D803689B688906CF
S31508000EF831EA030314BF0120002070470020704719
S31508000F08F0B590F82040013C012C6BD8066841B929
S31508000F18F468A40707D1436A43F40013436201201F
S31508000F2855E03469F5E70C013519D5F8B07107F0BD
S31508000F3804079760002F4BD1D5F8B0717F0D17605D
S31508000F48D5F8B07107F00207D760D5F8B47107F07D
S31508000F580F071761D5F8B471D5F8B4512644C7F305
S31508000F6807272D0C97615561D6F8B8211A700268BB
S31508000F782244D2F8B821120A5A7002682244D2F8D2
S31508000F88B821120C9A7002682244D2F8B821120EB7
S31508000F98DA7002682244D2F8BC211A71026822441F
S31508000FA8D2F8BC21120A5A7102682244D2F8BC2126
S31508000FB8120C9A7102681444D4F8BC21120EDA711C
S31508000FC8036851B9DA6842F02002DA600020F0BDF9
S31508000FD8D5F8B071FF085760B2E71A6942F02002DF
S31508000FE81A61F3E7436A43F4802397E7074AD36805
S31508000FF823F4E0631B041B0C43F0BF63000243F4AD
S31508001008003300F4E0600343D360704700ED00E066
S31508001018174B70B5DC68C4F30224C4F10705042D20
S3150800102804F1040328BF04254FF0FF36062B06FAF9
S3150800103805F38CBF033C002421EA0303A34006FA00
S3150800104804F422EA0404002843EA0403A8BF00F1CA
S3150800105860404FEA0313BCBF00F00F00054ADBB235
S31508001068AABF00F56140135480F8003370BD00BF6D
S3150800107800ED00E014ED00E00138B0F1807F0AD2F7
S31508001088064B074A5860F02182F8231000200722E9
S3150800109898601A6070470120704700BF10E000E0AA
S315080010A800ED00E0094910B50C6924F440740C6198
S315080010B80C6944F440740C610C6944F001040C6131
S315080010C80260BFF36F8F436010BD00BF003C02404B
S315080010D8074B1A6922F440721A611A6942F40072B7
S315080010E81A611A6942F001021A610160704700BF65
S315080010F8003C0240074B1A6922F440721A611A69C1
S3150800110842F480721A611A6942F001021A61018072
S31508001118704700BF003C02401A4BDA68D20606D56B
S315080011281949CA6942F01002CA611022DA60DA68F7
S31508001138900606D51449CA6942F00802CA612022EF
S31508001148DA60104BDA68510606D50F49CA6942F0C3
S315080011580402CA614022DA60DA68120606D50A4924
S31508001168CA6942F00202CA618022DA60054AD3686F
S315080011789B0706D50449CB6943F02003CB610223B4
S31508001188D3607047003C02405C1A0020064B1A6977
S31508001198002ABFBF054A5A6002F188325A60BABFA8
S315080011A81869C00F00207047003C024023016745B4
S315080011B8034A136943F0004313610020704700BFD0
S315080011C8003C0240F8B5124B124C00220546DA617B
S315080011D803F0FCF926460746E368DA030CD4E36805
S315080011E8DB0744BF0123E360F06810F0F20007D07C
S315080011F8FFF792FF012003E0691CEDD00DB9032023
S31508001208F8BD03F0E3F9C01BA842E5D9F7E700BF24
S315080012185C1A0020003C02402DE9F0411F4D984613
S315080012282B7E012B07460E46144635D001234CF271
S3150800123850302B76FFF7C6FFB0B9CFB9184B1A69E5
S3150800124822F440721A611A691A611A69E4B242F0FC
S3150800125801021A6134704CF25030FFF7B3FF104A96
S31508001268136923F00103136100232B76BDE8F08187
S31508001278012F04D1A1B23046FFF73CFFEBE7022F56
S3150800128804D121463046FFF723FFE4E722464346C2
S315080012983046FFF707FFDEE70220E7E75C1A00207B
S315080012A8003C0240074B1A6922F440721A611A690F
S315080012B842F004021A611A6942F4803242EA0020AE
S315080012C818617047003C024039B101291CD002292F
S315080012D80CBF4FF400714FF440710D4B1A6922F494
S315080012E840721A611A69114319611A6922F0F802DB
S315080012F81A611A6942F0020242EAC00018611A69BC
S3150800130842F480321A6170474FF48071E5E700BFEE
S31508001318003C0240144B1A6891050FD51A6822F446
S3150800132800721A601A6842F400621A601A6822F48F
S3150800133800621A601A6842F400721A600A4B1A6840
S3150800134852050FD51A6822F480621A601A6842F4A0
S3150800135880521A601A6822F480521A601A6842F48F
S3150800136880621A60704700BF003C02402DE9F843C6
S31508001378234E337E012B044688463FD001234CF280
S3150800138850303376FFF71EFF0546A8B94FF0FF33EE
S31508001398C8F800302368012B13D1207CFFF782FF99
S315080013A84CF25030FFF70EFF164A136923F0040370
S315080013B805461361FFF7AEFF002333762846BDE8D6
S315080013C8F883A768DFF83C90D4E902231344BB42A4
S315080013D8F0D9217C3846FFF777FF4CF25030FFF7F3
S315080013E8F1FED9F8103023F0FA03C9F8103018B10D
S315080013F8C8F800700546DDE70137E5E70225DDE7A9
S315080014085C1A0020003C02402DE9F04F85B00B68B5
S31508001418DFF8AC81684ADFF8AC9101930023012410
S31508001428019D9C402540AC4240F0B0804C6824F0B1
S31508001438100C4FEA430E03260CF1FF3706FA0EF690
S31508001448012F6FEA060611D8876807EA060ACF68E1
S3150800145807FA0EF747EA0A078760476827EA050A78
S31508001468C4F300179F4047EA0A074760C76807EAB0
S31508001478060A8F6807FA0EF747EA0A07BCF1020F49
S31508001488C76016D14FEAD30A00EB8A0A03F0070B9E
S31508001498DAF820704FEA8B0B4FF00F0C0CFA0BFC9E
S315080014A827EA0C0C0F6907FA0BF747EA0C07CAF87C
S315080014B8207007683E4004F0030707FA0EFE4EEA56
S315080014C806060660E60061D54FF0000BCDF80CB0AD
S315080014D8D8F84470394E47F48047C8F84470D8F8A5
S315080014E8447007F480470397039F23F0030707F11F
S315080014F8804707F59C3703F0030ED7F808A04FEA8C
S315080015088E0E4FF00F0C0CFA0EFCB0422AEA0C0CA1
S3150800151843D006F58066B04241D006F58066B042EB
S315080015283FD006F58066B0423DD006F58066B042E3
S315080015383BD048453BD006F50066B04239D006F59B
S315080015488066B04214BF0826072606FA0EF646EA4B
S315080015580C06BE601668EF4314F4803F0CBF3E4085
S315080015682E431660566814F4003F0CBF3E402E43BF
S315080015785660966814F4801F0CBF3E402E4396604A
S31508001588D668A40254BF3E402E43D6600133102BBA
S315080015987FF445AF05B0BDE8F08F5E46D5E701266E
S315080015A8D3E70226D1E70326CFE70426CDE70526A3
S315080015B8CBE70626C9E700BF003C01400000024009
S315080015C800380240001402402DE9F04F404DDFF87C
S315080015D80891DFF808A1DFF808B10022012303FA09
S315080015E802FE0EEA0104A6455FD122F0030606F1BB
S315080015F8804606F59C3602F0030C364BD6F808806A
S315080016084FEA8C0C0F2707FA0CF7984207EA0808DE
S3150800161850D003F5806398424ED003F5806398420C
S315080016284CD003F5806398424AD003F58063984204
S3150800163848D0484548D0504548D058450CBF072398
S31508001648082303FA0CF3434510D12B68E4432340D7
S315080016582B606B6823406B60AB682340AB60EB6814
S315080016681C40EC60B36823EA0707B76056000323F3
S315080016780468B340DB431C400460D40800EB8404C8
S3150800168802F0070C266A4FEA8C0C0F2707FA0CF7A4
S3150800169826EA07072762C4681C40C460446824EA27
S315080016A80E0444608468234083600132102A95D169
S315080016B8BDE8F08F0023C4E70123C2E70223C0E789
S315080016C80323BEE70423BCE70523BAE70623B8E7DE
S315080016D8003C014000000240001402400018024085
S315080016E8001C0240F0B504468BB060B390F8BD33D1
S315080016F8056803F0FF021BB980F8BC23FFF736F923
S31508001708032384F8BD33EB6B254613F4807355F829
S31508001718100B08BF236101F063F80FCD6E460FC69C
S315080017280FCD0FC695E8030086E803002546271D52
S3150800173897E80E0055F8100B00F098FF064620B1FA
S31508001748022384F8BD33012550E00146206801F0DC
S315080017584DF83046D4F804C01C264FF0010E014651
S31508001768C2B2944500F101001CD800231C2619466C
S31508001778D8B2844503F1010322D80FCD6E460FC6A9
S315080017880FCD0FC695E8030086E8030097E80E0014
S31508001798206801F06DF80123054600B3022284F893
S315080017A8BD23D0E706FB0243C3E9111183F83DE0E0
S315080017B883F83C20A3F8422083F83F101965CFE741
S315080017C806FB004282F8FD1182F8FC0182F8FF1137
S315080017D8C2F80412C2F80812C2F81012C8E784F848
S315080017E8380084F8BD33206801F098FB28460BB00A
S315080017F8F0BD38B5044610B90125284638BD032377
S3150800180880F8BD33006801F04BFB05460028F3D184
S315080018182046FFF7E5F884F8BD53EEE790F8BC33A1
S31508001828012B10B5044616D00123006884F8BC338A
S31508001838A36A012B06D1A369012B1EBF836B43F448
S315080018488033836300F0C6FF206801F059FB002047
S3150800185884F8BC0310BD0220FCE738B590F8BC3301
S31508001868012B04461BD00568012380F8BC3328469B
S3150800187800F0B6FF206801F051FB1021206800F03F
S31508001888CDFFA36A012B06D1A369012B1EBFAB6B3B
S3150800189823F48033AB63002084F8BC0338BD0220E8
S315080018A8FCE700002DE9F04F056887B0044628468E
S315080018B801F071FB0290002840F02181206801F0B0
S315080018C83BFB002800F01B81206801F035FB8207E6
S315080018D848BF2268206842BF536903F00203536170
S315080018E801F02AFBC3062AD52268936923F0100358
S315080018F893612E6AC6F34343022B06F00F0840F09D
S31508001908018147F6F0731E4214D01C2707FB0847C7
S31508001918C6F30A163246D7F80812284601F05EFAC0
S31508001928D7F808323344C7F80832D7F814321E44B1
S31508001938C7F814622268936943F010039361206814
S3150800194801F0FAFA070300F1EC80206801F0F4FACE
S3150800195846030BD5206801F0FBFA2646824600277F
S3150800196805F51069BAF1000F40F08981206801F081
S31508001978E3FA002815DAD5F8043823F00103C5F880
S31508001988043894F8F433012B40F01482002184F8C3
S31508001998F413204600F0D2FB2268536903F000438B
S315080019A85361206801F0C8FA01050BD5D5F808383F
S315080019B8DA0702D5204605F06FFB2268536903F457
S315080019C800635361206801F0B7FAC30435D505F5F5
S315080019D800667368206823F001037360102100F01D
S315080019E81DFF606805F510634FF67F31029A90422D
S315080019F840F0E481F36943F00113F361236B002B8C
S31508001A0800F0F881D6F8843043F00B03C6F8843022
S31508001A18736C43F00B037364D5F80038217C20688F
S31508001A2823F4FE63C5F8003804F5717201F0C8FAA4
S31508001A382268536903F480535361206801F07CFADD
S31508001A48870416D5206801F0AAFA206800F0CAFFAC
S31508001A58E060256800F074FB227B0146284600F002
S31508001A6845FE204605F007FB2268536903F4005330
S31508001A785361206801F060FA060707D5204605F085
S31508001A88F6FA2268536903F008035361206801F0DF
S31508001A9853FAC50208D50021204605F025FB226819
S31508001AA8536903F480135361206801F045FA8002EC
S31508001AB808D50021204605F013FB2268536903F46C
S31508001AC800135361206801F037FA410007D520460C
S31508001AD805F00EFB2268536903F0804353612068BA
S31508001AE801F02AFA42070AD523685D686B0702D50A
S31508001AF8204605F008FB226853682B43536007B055
S31508001B08BDE8F08F062B7FF415AF082204F571712E
S31508001B1828461C2701F062F907FB0847C6F30A1688
S31508001B2803E72068DFF8E492DFF8E4B201F008FA80
S31508001B3800268046B8F1000F3FF407AF18F0010FEA
S31508001B4861D05FFA86FA5146206801F009FA074615
S31508001B58F8071CD5730105F530621A442068012177
S31508001B68916000F530622169D0F840C01344012914
S31508001B789A686DD1110706D5CC4508D9100406D53B
S31508001B884FF4004202E0910641D520229A603807B0
S31508001B9820D5730105F530621A4408219160226838
S31508001BA8D2F840A002F530621344CA459A6804D9A7
S31508001BB8110444BF4FF400429A60204605F040FAE3
S31508001BC8CA4507D92169012904D104F57172206823
S31508001BD801F0F6F9FA0641BF05F5306303EB46133B
S31508001BE810229A60BB0641BF05F5306303EB46131E
S31508001BF820229A60B80441BF05F5306303EB461303
S31508001C084FF400529A6001364FEA580892E712F0E4
S31508001C18280FBCD1CC4501D91204B1D41C2202FB29
S31508001C2806421B69D2F80412C3F31203CB1AC2F888
S31508001C381432D2F808321944C2F8081286B9D4F808
S31508001C4810326BB904F57172012101F0B9F907E090
S31508001C58DC450AD1110493D4920601D520229A604C
S31508001C685146204605F0F2F991E7002EF8D1D4F846
S31508001C781032002BF4D104F571723146E5E71AF0F3
S31508001C88010F74D05FFA87FB5946206801F071F98D
S31508001C9810F0010F804620D0D5F834382169012084
S31508001CA807F00F0200FA02F223EA0203C5F83438ED
S31508001CB809EB4713814298600BD1D6E911231344DF
S31508001CC8B36437B9236D23B904F57172206801F036
S31508001CD877F95946204605F0C2F918F0080F1EBFCD
S31508001CE809EB471308229A6018F0100F1EBF09EB74
S31508001CF8471310229A6018F0400F1EBF09EB4713C6
S31508001D0840229A6018F0020F1EBF09EB47130222F9
S31508001D189A6018F0800F2AD0D6E914329A4226D843
S31508001D289B1A726C21680391934228BF13460333A2
S31508001D389B08049301F5106303EB47130593059B6A
S31508001D480498996989B28142D6E9143214D2934221
S31508001D580DD8039B07F00F0203F5006B0121D3F892
S31508001D68343801FA02F223EA0203CBF83430013791
S31508001D784FEA5A0A1C36F5E59342EAD9002BE8D009
S31508001D88A3EB0208736C0398984528BF984608F190
S31508001D9803039B080493237C00935A461FFA88F387
S31508001DA8B16C00F02FFFB36C4344B364736D4344BE
S31508001DB87365C4E7204605F089F9EDE599601A6860
S31508001DC822F400121A601A6842F000621A60C3F810
S31508001DD80812D3F8002222F40012C3F80022D3F816
S31508001DE8002242F00062C3F80022029A01320292E7
S31508001DF82033FBE5736943F4005343F02B037361FF
S31508001E08336943F00B03336106E600BF0A30544FC3
S31508001E180A31544F90F8BC33012B10B5044613D039
S31508001E280123006884F8BC33A36A012B06D1A36989
S31508001E38012B1EBF836B43F48033836301F060F87C
S31508001E48002084F8BC0310BD0220FCE738B590F8DA
S31508001E58BC33012B044614D00568012380F8BC332B
S31508001E68284601F05BF8A36A012B06D1A369012B62
S31508001E781EBFAB6B23F48033AB63002084F8BC0326
S31508001E8838BD0220FCE790F8BC23012A10B50446A1
S31508001E980BD0012280F8BC2384F83810006801F0BA
S31508001EA81FF8002084F8BC0310BD0220FCE770B5B3
S31508001EB801F00F05044611F0800FC5EBC5004FEA7F
S31508001EC880004FF01C061FD006FB054600F13C01B2
S31508001ED80120214486F83D008A604A780D70CB7047
S31508001EE802B1CD80022B04BF00230B7194F8BC33D2
S31508001EF8012B12D0012384F8BC33206800F07DFD3D
S31508001F08002084F8BC0370BD06FB054600F5FE7183
S31508001F180020214486F8FD01DEE70220F3E710B524
S31508001F28044601F00F00C0EBC00311F0800F4FEA1A
S31508001F3883034FF01C0216D002FB004203F13C0152
S31508001F480123214482F83D30087094F8BC33012BEC
S31508001F5812D0012384F8BC33206800F08DFD0020D8
S31508001F6884F8BC0310BD02FB004203F5FE7100238A
S31508001F78214482F8FD31E7E70220F3E738B501F096
S31508001F880F051C2404FB050104FB050401F5FE7175
S31508001F98C4F810320023C4F80822C4F8143284F8A6
S31508001FA8FD3184F8FC5103690068012B08BFC4F8A1
S31508001FB80C22DAB21DB900F0B1FD002038BD00F0D8
S31508001FC835FEFAE71C2301F00F0103FB0101D1F8DE
S31508001FD81402704738B501F00F051C2404FB0501E7
S31508001FE804FB05043C312365002363650123A264C9
S31508001FF884F83D3084F83C5003690068012B08BF13
S31508002008E264DAB21DB900F089FD002038BD00F097
S315080020180DFEFAE738B5436801F00F059D420446F8
S315080020282ED811F0800F4FF01C021FD002FB0501B5
S3150800203802FB050301223C3381F83D2001229A70F0
S315080020481D7094F8BC1391421CD084F8BC23194619
S31508002058206800F0D1FE2DB904F57172217C20683C
S3150800206800F0AEFF002084F8BC0338BD02FB01036C
S3150800207802FB0101002203F5FE7381F8FD21DDE765
S315080020880120F2E70220F0E738B5436801F00F02AD
S315080020989A4204462AD8C2EBC20311F0800F4FEAC7
S315080020A883034FF01C0018D000FB024003F13C01E3
S315080020B80123214480F83D3000258D700A7094F874
S315080020C8BC33012B14D0012384F8BC33206800F0F4
S315080020D8BEFE84F8BC53284638BD00FB024003F50B
S315080020E8FE710023214480F8FD31E5E70120F3E776
S315080020F80220F1E7006870B51204446A19B9224348
S315080021088262002070BD836A4D1E04EB13440023C7
S315080021185E1CDBB29D4205D83F3100EB81002243A5
S315080021284260EEE7403300EB83035B6804EB134435
S315080021383346EDE703680020596270477047000088
S31508002148014B1868704700BF00000020024A13694F
S3150800215818431061704700BF00380240024A1369E5
S3150800216823EA0000106170470038024008B5274B7B
S31508002178984207D10120FFF7E9FF0120FFF7EEFF94
S31508002188002008BD224B984204D10220FFF7DEFF43
S315080021980220F3E71F4B984204D10420FFF7D6FF25
S315080021A80420EBE71C4B984204D10820FFF7CEFF22
S315080021B80820E3E7194B984204D11020FFF7C6FF19
S315080021C81020DBE7164B984204D12020FFF7BEFF04
S315080021D82020D3E7134B984204D14020FFF7B6FFD7
S315080021E84020CBE7104B984204D18020FFF7AEFF7A
S315080021F88020C3E70D4B984206D14FF48070FFF74D
S31508002208A5FF4FF48070B9E70120BAE7000002403D
S315080022180004024000080240000C02400010024078
S315080022280014024000180240001C02400020024028
S315080022382DE9F04F02460D6895FAA5F44FF0010E00
S31508002248B4FA84F403264FF00F0C35FA04F001D1DA
S31508002258BDE8F08F0EFA04F32B406DD04868471E88
S31508002268012F1ED8976893FAA3F8B8FA88F893FA4C
S31508002278A3F94FEA480806FA08F827EA0808B9FA4F
S3150800228889F98F684FEA490907FA09F748EA0707F3
S315080022989760576827EA0308CF685F4348EA07073D
S315080022A85760D76893FAA3F8B8FA88F893FAA3F99F
S315080022B84FEA480806FA08F827EA0808B9FA89F929
S315080022C80F694FEA490907FA09F748EA070702288A
S315080022D8D7601DD193FAA3F7B7FA87F7072FD1F86E
S315080022E814A02BDC176A93FAA3F9B9FA89F993FAB1
S315080022F8A3F8B8FA88F84FEA89090CFA09F94FEAEF
S31508002308880827EA09070AFA08FA47EA0A07176245
S31508002318D2F8008093FAA3F7B7FA87F793FAA3F3E4
S31508002328B3FA83F37F0006FA07F75B0028EA07077C
S3150800233800FA03F33B431360013486E7D2F824B066
S315080023481F0A97FAA7F8B8FA88F897FAA7F7B7FA0C
S3150800235887F74FEA88080CFA08F8BF002BEA080B33
S315080023680AFA07F74BEA07075762D1E7214B1A68B3
S3150800237842F0010282B01A601A689207FCD5002258
S315080023889A601A680192019A22F0867222F48032BB
S315080023980192019A22F080620192019A1A601A68DB
S315080023A822F0F80242F080021A60124B186810F000
S315080023B80070FBD1104A5A60104AC3F88420DA68BC
S315080023C822F4F852DA60DA6822F40052DA60DA6837
S315080023D842F41F02DA60DA6842F40012DA605A6FC9
S315080023E822F001025A675A6F42F080725A6702B0A1
S315080023F8704700BF00380240103000240030002023
S31508002408034B044A9B68C3F30313D35CD84070474D
S3150800241800380240D1730008034B044A9B68C3F38B
S315080024288223D35CD840704700380240E17300081D
S31508002438034B044A9B68C3F34233D35CD8407047BE
S3150800244800380240E17300080F4B104A596810B566
S315080024580F4C01F48001002908BF2246082810D12C
S31508002468596858685B68C3F30143C0F38810013399
S3150800247801F03F015B00B2FBF1F25043B0FBF3F009
S3150800248810BD0020FCE700BF0038024000127A00A1
S315080024980024F400064B986800F00C00042803D0C2
S315080024A8082803D00348704703487047FFF7CCBF8E
S315080024B8003802400024F40000127A0010B50446D9
S315080024C8FFF7E8FF2060FFF79BFF6060FFF7A4FFB0
S315080024D8A0606068FFF7ACFFE06010BD026812F004
S315080024E84002F0B5044624D1D1E900373B438F684A
S315080024F84D690668086A3B43CF683B430F693B4307
S315080025088F692B433B43CF6926F47F463B430343F6
S3150800251826F0BF0633432360636823F0040343EABF
S315080025281545B0F5005F656001D18B8C23611046AF
S3150800253800E00120E36923F40063E361F0BD0000CD
S315080025487FB5C3689B0404460D4602D5012004B02E
S3150800255870BD4B68C968C2680B4329690B43A969EA
S3150800256822F416420B4322F00C021343C360036994
S31508002578AA6823F440531343036143696A6923F439
S315080025884073134343616846FFF798FF284B9C42FC
S3150800259829D103980028D9D02B68002BD6D0192220
S315080025A8A0FB0201AA69B2F5004F31D1DA184FF03B
S315080025B8000646EB0603FDF703FE6421B0FBF1F5BA
S315080025C801FB1503DB003233B3FBF1F39BB203F0CF
S315080025D807025B0002EB051203F4F87313449BB277
S315080025E8A3600020B3E7134B9C4201D10298D1E7B8
S315080025F8114B9C42FAD003F54C439C42C9D0A3F52B
S3150800260848439C42F2D003F580639C429ED1EDE78D
S315080026189A009B0FFDF7D4FD6422B0FBF2F102FB8A
S3150800262811031B013233B3FBF2F303EB0113D6E7AD
S315080026380010014000440040004800400A4B013B96
S315080026480FD00269002AFADA0369074A43F0010338
S315080026580361013A05D0036913F00103F9D1184655
S3150800266870470320704700BF410D030084B038B592
S3150800267805AD85E80E000A9B012B044625D1836B18
S3150800268823F480338363C36823F4840323F0400365
S31508002698C360C36823F44013C360119B012B02BFB0
S315080026A8C36843F48013C360FFF7C8FF089B012B70
S315080026B807D1A36843F00603A360A36843F0200381
S315080026C8A360BDE8384004B07047C36843F04003C8
S315080026D8C360FFF7B3FF0E9B23B9A36B43F480339C
S315080026E8A363E3E7A36B23F48033F9E7022A58D1F7
S315080026F82E4B2F4A0B44934247D92E4B2E4A0B444E
S31508002708934244D9A1F574032C4AA3F5105393426E
S315080027183FD9A1F1837302F5C332A3F5E743A03283
S31508002728934238D9264B274A0B44934235D9264B28
S3150800273802F592220B4402F5787293422FD9234B5D
S3150800274802F5C3220B4402F52072934229D9A1F156
S31508002758B77302F5B712A3F5585302F558729342A0
S3150800276821D91B4B02F512220B4402F5F862934253
S3150800277894BF07230623C26822F47052C260C2684F
S3150800278842EA8323C360002070470F23F3E70E232A
S31508002798F1E70D23EFE70C23EDE70B23EBE70A2315
S315080027A8E9E70923E7E70823E5E700BF405327FFDA
S315080027B8FF340C00401E1BFF3F420F007F4F1200DC
S315080027C860B6E5FE5FE3160000D3CEFEC05BB3FE37
S315080027D8E05459FE836843F001038360002070477C
S315080027E8836823F0010383600020704708B5C3682F
S315080027F8012923F0C043C36008D1C36843F00053D6
S31508002808C3603220FEF7E0F9002008BD19B9C3688D
S3150800281843F08043F4E70120F7E70000890141F017
S315080028282001064A0161013A05D0036913F020031D
S31508002838F9D1184670470320704700BF410D0300B9
S315080028481023064A0361013A05D0036913F01003F9
S31508002858F9D1184670470320704700BF410D030099
S31508002868D0F800381943C0F800180020704700004F
S3150800287884B02DE9F843044609A880E80E00002329
S31508002888139D0F46194603F1400204EB82020133F1
S315080028980F2B5160F7D104F50066002D6CD17368CB
S315080028A843F002037360A36B43F40013A363A36B9B
S315080028B823F40023A363A36B23F48023A3630023D1
S315080028C8C4F8003ED4F80038C4F800380E9B012B2B
S315080028D85CD10B99002957D12046FFF7C1FF102173
S315080028E82046FFF79BFF01462046FFF7A9FF002869
S315080028F84ED1081C18BF01200023336104F5106265
S3150800290873611946F3614FF0904C4FF0006E4FF61D
S315080029187F38BB423ED1002104F530620F464FF09E
S31508002928904C4FF0006E4FF67F388B4245D133698D
S3150800293823F4807333610023A3616FF080436361D6
S315080029480C9B1BB9A36943F01003A361A269244B26
S315080029581343A3610F9B1BB1A36943F00803A36143
S31508002968012D01BFA36943F0804343F00403A36123
S31508002978BDE8F84304B07047A36B23F40013A363B8
S31508002988A36B43F4002399E71946A5E70321A3E7B0
S315080029980120B1E7D2F80090B9F1000F0BDA3BB97C
S315080029A8C2F800E011610133C2F808802032B0E7A6
S315080029B8C2F800C0F6E71160F4E7D2F80090B9F15A
S315080029C8000F0BDA39B9C2F800E017610131C2F80D
S315080029D808802032A9E7C2F800C0F6E71760F4E7CE
S315080029E800383C80D0F8083813F0060004D013F0F5
S315080029F8020F14BF02200F20704730B50D78012446
S31508002A0805F00F039C404B7800F50062012B00EB9C
S31508002A184510D36918D11C43D461D0F800391A0473
S31508002A2810D48B68C978D0F80029C3F30A0343F091
S31508002A38805343F4004343EA814343EA85531343E7
S31508002A48C0F80039002030BD43EA0444D461D0F800
S31508002A58003B1B04F6D48B68C978D0F8002BC3F35F
S31508002A680A0343F0805343F4004343EA814313437C
S31508002A78C0F8003BE6E7000010B50A78497801294E
S31508002A8800EB421302F00F0100F5006020D1D3F8DD
S31508002A980029002A0BDAD3F8002942F00062C3F8A5
S31508002AA80029D3F8002942F08042C3F800290122F8
S31508002AB8C46B8A40D2431440C463C1690A40C261E0
S31508002AC8D3F80019134A0A40C3F80029002010BD94
S31508002AD8D3F8002B002A0BDAD3F8002B42F0006251
S31508002AE8C3F8002BD3F8002B42F08042C3F8002B1A
S31508002AF84FF48032C46B8A40D2431440C463C16918
S31508002B080A40C261D3F8001B034A0A40C3F8002BDF
S31508002B18DCE700BF007833EC0078F3EF4B78F0B5C4
S31508002B280C784D69354E364F012B00EB441444D1C9
S31508002B3804F51063B5B91D692E401E611D6945F473
S31508002B4800251D611D692F401F61012A21D10A69C7
S31508002B5802B15A61D4F8003943F00443C4F800397D
S31508002B680020F0BDD3F810C00CEA07071F611F69DB
S31508002B783E401E618E68AE421D6938BF4E6145F4F7
S31508002B8800251D614D691E69C5F3120535431D618A
S31508002B98DBE7D4F8003943F00443C4F800394B6935
S31508002BA8002BDDD00B78D0F8344803F00F02012348
S31508002BB893402343C0F83438D2E704F530631869DC
S31508002BC838401861186930401861886805B1486145
S31508002BD81D6945F400251D611D69C0F312002843C7
S31508002BE8012A186102D1CA6802B15A61D4F8003BB1
S31508002BF843F00443C4F8003BB2E700BFFFFF07E011
S31508002C080000F8FF10B59DF808404CB9033300EBEF
S31508002C1802309B0800F5805001EB8303994201D1E5
S31508002C28002010BD51F8042B0260F7E7F7B54D7878
S31508002C380C784B69CE78DFF89CC1DFF89CE1012D4A
S31508002C4800EB44147CD104F510652F693BBB07EAF1
S31508002C580C072F612F6947F400272F612F6907EAA8
S31508002C680E072F61012A41D10B6903B16B61012E49
S31508002C780CD1D0F8083813F4807FD4F800390CBF83
S31508002C8843F0005343F08053C4F80039D4F80039A8
S31508002C9843F00443C4F80039002003B0F0BD07EA3E
S31508002CA80E072F612F6907EA0C07D1F808C02F61AC
S31508002CB80CEB0307013FB7FBFCFC454FD5F810E0C2
S31508002CC807EACC4747EA0E072F61D5F810C0C3F3C1
S31508002CD8120747EA0C07012E2F61C3D12F6927F07F
S31508002CE8C0472F612F6947F00057BAE7D4F800594B
S31508002CF8012E45F00445C4F800590CD0002BCBD05A
S31508002D080B78D0F8344803F00F0201239340234385
S31508002D18C0F83438C0E7D0F8085815F4807FD4F8D6
S31508002D2800590CBF45F0005545F08055C4F80059C0
S31508002D380C7800929BB22246C968FFF763FFABE797
S31508002D4804F530673D6905EA0E053D613D6905EA02
S31508002D580C053D618D681BBB3B69C5F312051D4310
S31508002D683D613B6943F40023012A3B6102D1CB68E4
S31508002D7803B17B61012E0CD1D0F8083813F4807F93
S31508002D88D4F8003B0CBF43F0005343F08053C4F813
S31508002D98003BD4F8003B43F00443C4F8003B7BE708
S31508002DA8DFF82CC0D7F810E02B44013BB3FBF5F34A
S31508002DB80CEAC34C4CEA0E0CC7F810C09BB2D7F8FD
S31508002DC810C06B43C3F3120343EA0C03CCE700BFF6
S31508002DD80000F81FFFFF07E00000F8FF033292081B
S31508002DE801EB820200F58050914201D108467047EE
S31508002DF8036841F8043BF7E74A780B78012A00EBA1
S31508002E08431012D1D0F80029002A06DB2BB1D0F8D6
S31508002E18003923F08043C0F80039D0F8003943F464
S31508002E280013C0F8003900207047D0F8002B002A94
S31508002E3806DB2BB1D0F8003B23F08043C0F8003BF3
S31508002E48D0F8003B43F40013C0F8003BEBE70B78D7
S31508002E584A7800EB4310CB78012AA3F10203DBB2C8
S31508002E680FD1D0F80029012B22F40012C0F8002946
S31508002E7805D8D0F8003943F08053C0F80039002047
S31508002E887047D0F8002B22F40012012BC0F8002B4B
S31508002E989EBFD0F8003B43F08053C0F8003BEEE7EE
S31508002EA810B500F51063044600F52E614FF67F321B
S31508002EB89A60C3F8082220338B42F9D10022C4F855
S31508002EC810282046C4F81428C4F81C28FFF7B8FCAC
S31508002ED828B920461021BDE81040FFF79FBC10BD51
S31508002EE8D0F8003823F4FE63C0F80038D0F8003864
S31508002EF8090101F4FE611943C0F80018002070475B
S31508002F08D0F8003E23F00303C0F8003ED0F8043892
S31508002F1823F00203C0F8043800207047D0F8003EB2
S31508002F2823F00303C0F8003ED0F8043843F0020340
S31508002F38C0F8043800207047426980691040704715
S31508002F48D0F8183800F50060C0691840000C7047BA
S31508002F58D0F8183800F50060C069184080B2704784
S31508002F6800EB411100F50060D1F8082B40691040C4
S31508002F78704710B5D0F81048D0F8343800EB41102F
S31508002F8801F00F01CB4000F51060DB018068DBB269
S31508002F982343184010BD406900F001007047D0F877
S31508002FA8003923F4FF6323F00703C0F80039D0F883
S31508002FB8043843F48073C0F80438002070470000CA
S31508002FC830B5056C104CA54200F5306303D9D0F826
S31508002FD8004B002C16DB00241C611C6944F40024F1
S31508002FE81C611C6944F018041C611C69012944F019
S31508002FF8C0441C6101BF5A61D0F8003B43F08023E6
S31508003008C0F8003B002030BD0A30544F014B186009
S31508003018704700BF0000002070B50A4D287301F0FC
S31508003028CDFA00F13206AC6814F0010407D101F0B4
S315080030385CFD01F0C3FAB042F5D9204670BDE868D0
S31508003048C0B2FBE700380040034B4FF480529A6140
S31508003058FF20FFF7E1BF00BF0004024038B501F0C2
S31508003068ADFA00F5FA75FF20FFF7D6FF044601F01A
S315080030783CFDFF2C03D001F0A1FAA842F3D3A4F132
S31508003088FF035842584138BD084B4FF0805210B5D7
S31508003098FF209A61FFF7C0FFFFF7E0FF044618B95B
S315080030A8FFF7D2FF204610BD0124FBE700040240C3
S315080030B8020670B504460E4608D500213720FFF7E4
S315080030C8F7FF0128054631D804F07F04FFF7BCFF4F
S315080030D8FFF7DAFF70B344F04000FFF79DFF300EA4
S315080030E8FFF79AFFC6F30740FFF796FFC6F30720D0
S315080030F8FFF792FFF0B2FFF78FFFCCB1082C14BF89
S3150800310801208720FFF788FF0C2C02D1FF20FFF744
S3150800311883FF0A24FF20FFF77FFF054601F0E5FC39
S315080031282B0603D5013C14F0FF04F3D1284670BDDD
S315080031389520E7E7FF25F9E738B5841C00F202254C
S3150800314814F8020CFFF768FF023414F8030CFFF7AB
S3150800315863FF01F0CAFCAC42F2D1FF20FFF75CFF1F
S31508003168FF20FFF759FFFF20FFF756FF00F01F0063
S31508003178431F5842584138BDF8B505460E4601F072
S315080031881DFA00F16407FF20FFF746FF044601F021
S31508003198ACFCFF2C05D101F011FAB842F3D3002094
S315080031A8F8BDFE2CFBD10236AC1C3544FF20FFF7D0
S315080031B833FF04F8020CFF20FFF72EFF023404F849
S315080031C8030C01F092FCAC42F0D1FF20FFF724FF74
S315080031D8FF20FFF721FF0120E2E700002DE9F04F65
S315080031E899B0002840F037819C4B1C7814F00204EB
S315080031F81D4604D01878C0B219B0BDE8F08F984BB0
S31508003208DFF864821A6B974E42F002021A631A6B49
S3150800321802F002020192019A1A6C42F480421A6478
S315080032281B6C069403F480434FF4805902274FF029
S31508003238010A009302A94046CDE9029ACDE9047429
S31508003248009BFEF7F5FF4FF46043C8F81890CDE9E0
S3150800325802370323CDE9043402A905234046069418
S315080032680793FEF7E5FF4FF48273CDE90F344FF461
S3150800327800713023CDE91313304607230EA90E949F
S31508003288CDE91144CDE915441793FFF727F9736873
S3150800329823F010037360336843F040033360C8F8BB
S315080032A81890CDE90A7408AF4FF4004939464046E4
S315080032B8CDE9089A0C94B246FEF7BAFF0A24C8F86C
S315080032C818904FF0FF0901F079F900F1640BB3681B
S315080032D89A0703D401F072F98345F8D28AF80C9054
S315080032E801F06CF900F1640BB368DB0703D401F04D
S315080032F865F98345F8D2013CE5D14FF4004002232D
S31508003308CDE908030323CDE90A3439460523564887
S315080033180D930C94FEF78CFF4FF08053C8F81830BD
S3150800332821462046FFF7C4FE0128064640F0848059
S3150800333801F044F94FF4D57100F57A780820FFF7BB
S31508003348B7FE012860D1FF20FFF766FE385501341D
S31508003358042CF8D19DF82230012B6DD19DF8233025
S31508003368AA2B69D101F02AF9404506D24FF08041C7
S31508003378A920FFF79DFE0028F4D101F01FF9404562
S315080033885AD200213A20FFF793FE002854D1044662
S31508003398FF20FFF741FE38550134042CF8D19DF873
S315080033A8203013F0400F14BF0C2404242F4B1C6044
S315080033B8FFF74AFE2B78002C49D02A4C03F0FE0367
S315080033C82B70236823F0400323604FF4827200238E
S315080033D8CDE90E324FF400710822CDE91033129365
S315080033E8CDE91312CDE915330EA9072320461793FD
S315080033F8FFF774F8636823F010036360236843F0E3
S31508003408400323602878F6E62146A920FFF750FEF0
S31508003418022836BF02240124A92601F0CFF8404520
S315080034280CD301F0CBF8404506D24FF400711020B2
S31508003438FFF73EFE0028B9D00024B7E7002130463A
S31508003448FFF736FE0028ECD001F04FFBE5E743F01E
S3150800345801032B70D6E70120CEE600BF0C0000203A
S31508003468003802400038004000040240CC0400201E
S3150800347818B9034B1878C0B270470120704700BFC7
S315080034880C00002038B50D461C46114698BB93B368
S315080034981B4B1B78DA0730D41A4B1B681B0758BF17
S315080034A84902012C11D11120FFF702FE38B94FF451
S315080034B800712846FFF760FEB0FA80F46409FFF742
S315080034C8C3FD201C18BF012038BD1220FFF7F0FDE8
S315080034D80028F4D14FF400712846FFF74DFE28B1AD
S315080034E801F003FB013C05F50075F3D100210C201A
S315080034F8FFF7DEFDE3E70420E6E70320E4E700BF7D
S315080035080C000020CC04002070B50D4616461C4653
S3150800351800284ED1002B4CD0294B1A78D0074AD40C
S315080035281B78590749D4274B1B681A0758BF7602D0
S31508003538012C19D131461820FFF7BAFD30B10124FC
S31508003548FFF782FD201C18BF012070BDFFF786FD16
S315080035580028F4D0FE20FFF75FFD2846FFF7ECFDAC
S31508003568B0FA80F46409EBE713F0060F03D0214696
S315080035789720FFF79DFD31461920FFF799FD00288A
S31508003588DED1FFF76BFD60B1FC20FFF745FD284645
S31508003598FFF7D2FD28B101F0A8FA013C05F5007538
S315080035A8EFD1FFF75BFD0028C9D0FD20FFF734FDF2
S315080035B8C6E70420C9E70320C7E70220C5E700BF16
S315080035C80C000020CC0400207FB51546002840F0E2
S315080035D8DF80714B1B78DA0700F1DC800E2900F2D0
S315080035E8D580DFE801F0080ED34FD3D3D3D3D3D38E
S315080035F89CA0ACAFC200FFF747FDB0FA80F4640997
S3150800360806E000210920FFF753FD044628B10124E6
S31508003618FFF71AFD204604B070BD10216846FFF76B
S31508003628ABFD0028F3D09DF800309DF808109DF8EA
S3150800363809009B09012B9DF8073009D11A0402F4E1
S315080036487C1200EB012101320A4492022A60DFE764
S315080036589DF806209B00920203EB911302F4406240
S3150800366813449DF805209DF80A1002F00F0202EB94
S31508003678D112410001F006010A440133073A934082
S315080036882B60C5E7454C216811F004011BD00021C1
S315080036988D20FFF70DFD0028B9D1FF20FFF7BCFCE8
S315080036A810216846FFF768FD0028B0D03024FF20AF
S315080036B8013CFFF7B1FC14F0FF04F8D19DF80A3075
S315080036C81A091023DBE70920FFF7F2FC00289ED128
S315080036D810216846FFF750FD002898D024689DF801
S315080036E80A309DF80B1014F002040DD05B009DF803
S315080036F80D2003F07E0303EBD11392090133013A37
S3150800370893402B60002483E7CA0002F01802C3F32B
S31508003718840302EB5112013302FB0333B0E71F4B54
S315080037281B682B70EEE700210920FFF7C1FC00286B
S315080037387FF46DAF10212846FFF71EFD5DE70021CF
S315080037480A20F2E700213A20FFF7B2FC00287FF4A6
S315080037585EAF6C1E0335FF20FFF75EFC04F8010F09
S3150800376801F0C3F9AC42F6D1CCE70C4B1B685B07F2
S315080037787FF54DAF00218D20FFF79AFC00287FF4CE
S3150800378846AFFF20FFF748FC4021D4E704243FE76B
S3150800379804243FE703243DE70C000020CC0400205E
S315080037A8A0B1D0F8B83213B10023C0F8B832D0F8AF
S315080037B8CC3213B10023C0F8CC3209B1C0F8B41220
S315080037C8012380F89C32027003F0A8BC03207047D6
S315080037D8012310B580F89C32D0F8B832044613B1E4
S315080037E85B6801799847D4F8CC3213B10023C4F83A
S315080037F8CC32204603F0E2FC20B92046BDE810404A
S3150800380803F0C0BC10BD37B500240546ADF8064020
S3150800381851B1C0F8B812CB6A0DF106009847C5F839
S31508003828CC02204603B030BD0320FBE703F0B8BC42
S31508003838D0F8B8320BB11B6818470320704708B58B
S31508003848D0F8B8320BB15B689847002008BD38B580
S31508003858044600F2AA25284600F00BFB012394F833
S31508003868AA12C4F89432B4F8B032C4F8983201F0FF
S315080038781F03012B0FD008D3022B12D0204601F0C4
S315080038888001BDE8384003F0C5BC29462046BDE896
S31508003898384000F0F5B829462046BDE8384000F01B
S315080038A82FBA29462046BDE8384000F050BA70B508
S315080038B80446164609BBD0F89432032B0ED1D0F825
S315080038C85C31D0F8602193420AD99B1A9A42C0F80B
S315080038D85C3128BF1A46314600F01BFB002070BD34
S315080038E8D0F8B8321B6923B190F89C22032A00D174
S315080038F89847204600F015FBF0E7D0F8B8329B69E0
S3150800390833B190F89C22032A02D1BDE870401847C3
S315080039180320E4E770B5044616460D46D9BBD0F829
S315080039289432022B0ED1D0E907239A4213D9D21A18
S31508003938C261314600F0E5FA2B462A462946204652
S3150800394803F0B4FC94F8A032012B4FF0000001D123
S3150800395884F8A00270BD0CD183699A4209D8D0F8B8
S315080039689822934205D20A4600F0CBFAC4F8985230
S31508003978E2E7D4F8B832DB682BB194F89C22032A1C
S3150800398801D1204698478021204603F043FC20466B
S3150800399800F0D2FAD6E7D0F8B8325B6933B190F8B6
S315080039A89C22032A02D1BDE8704018470320D1E7B4
S315080039B8012370B580F89C32D0F8BC320021044641
S315080039C8C0F894124160C0F8A4121BB1D0F8B832F6
S315080039D85B68984700224025114601264023204661
S315080039E803F0FAFBA4F86461C4F860512B46002278
S315080039F88021204603F0F0FBA6842562002070BDCE
S31508003A0801740020704790F89C3280F89D32042390
S31508003A1880F89C320020704790F89C32042B04BF2B
S31508003A2890F89D3280F89C320020704708B590F8C7
S31508003A389C22032A04D1D0F8B832DB6903B1984727
S31508003A48002008BD002070470020704700207047F6
S31508003A58012208B580F89C22D0F8B82212B152681B
S31508003A6801799047002008BD10B58021044603F067
S31508003A78D1FB20460021BDE8104003F0CBBB00006F
S31508003A88F7B50B7803F06003202B04460E4612D0D0
S31508003A98402B10D0002B58D14B78092B55D8DFE886
S31508003AA813F000011E01540015015400810014008A
S31508003AB85400E900A000D4F8B83231469B6820467D
S31508003AC898470546284603B0F0BD0023ADF80630EA
S31508003AD84B881A0A013A062A37D8DFE802F0041C86
S31508003AE82936364E5800D0F8B4321B68207C0DF1BA
S31508003AF806019847F288002A00F0ED80BDF80630DE
S31508003B081BB39A4228BF1A46ADF806200146204636
S31508003B1800F0EAF95FE0027CD0F8B83232B99B6A5D
S31508003B280DF10600984702234370E3E7DB6AF7E7D7
S31508003B38DBB2052B09D8DFE803F0030C1014181CB0
S31508003B48D0F8B4325B68002BD0D12046FFF78CFF3B
S31508003B5841E0D0F8B4329B68F5E7D0F8B432DB68B0
S31508003B68F1E7D0F8B4321B69EDE7D0F8B4325B69EF
S31508003B78E9E7D0F8B4329B69E5E7037C002BE4D182
S31508003B88D0F8B8320DF106005B6B9847B2E7037CAC
S31508003B98002BDAD1D0F8B8320DF106001B6B98471E
S31508003BA80723C1E78B88002BCFD1CF88002FCCD12C
S31508003BB84D887F2DC9D890F89C32032BC5D0E9B219
S31508003BC880F89E1203F056FB204600F0AAF925B1A4
S31508003BD8022384F89C32002574E7012384F89C3272
S31508003BE870E78D78454E012D357003D9FFF73CFFF0
S31508003BF8032567E790F89C32022B08D0032B16D0CA
S31508003C08FFF732FF31782046FFF719FEF0E7002D57
S31508003C1861D001214160FFF70BFE0546204615B124
S31508003C28FFF722FF4EE700F07CF90323D6E755B9DC
S31508003C38022380F89C3245602946FFF700FE204695
S31508003C4800F06FF93EE74168012944D0C9B2FFF789
S31508003C58F6FD317861602046FFF7EAFD054600283B
S31508003C6839D02046FFF700FF21792046FFF7E7FD00
S31508003C780223B3E7CA88012A7FF467AF90F89C3213
S31508003C88002B3FF462AF022B04D9032B7FF45DAFF8
S31508003C98011D3CE70146002541F8085F00F024F9B4
S31508003CA810E790F89C32013B022B3FF64EAFCB88C3
S31508003CB8022B7FF44AAF0123C360D0F8A4320BB1B4
S31508003CC80323C360022204F10C0120E74B88012B69
S31508003CD881D1C0F8A432204600F023F97BE790F892
S31508003CE89C32013B022B3FF630AF4B88012B4FF035
S31508003CF800057FF4E7AEC0F8A452A0E7D004002078
S31508003D0870B50B7803F06003202B04460E4602D0E4
S31508003D18402B00D0B3B994F89C32013B022B11D83A
S31508003D283379012B0ED8D4F8B83231469B68204629
S31508003D389847F38805461BB910B9204600F0F1F8EC
S31508003D48284670BD2046FFF78FFE0025F8E770B5B0
S31508003D580B7803F06003202B04460D4614D0402B3D
S31508003D6812D06BB96A788B88012AD9B221D040D388
S31508003D78032A05D190F89C32022B31D0032B0BD09D
S31508003D882046FFF771FE12E0D4F8B83229462046D5
S31508003D989B68BDE8704018476B882BB94A0603D05C
S31508003DA8EB880BB903F036FA204600F0BAF800207B
S31508003DB870BD90F89C32022B12D0032BE0D16B8889
S31508003DC8002BF4D14E0601D003F032FA204600F053
S31508003DD8A8F8D4F8B83229469B6820469847E6E7F3
S31508003DE84B06CDD003F016FA8021204603F012FAC6
S31508003DF8DDE790F89C22022A19D0032AC0D101F0DF
S31508003E080F0213F0800F4FF0140303FB02021DD0B4
S31508003E18928C002AB4D001F07F0505FB03350544CA
S31508003E2811F07F031DD12B60022229460AE04A06B3
S31508003E38A6D11B064CBF00F1140100F5AA71002390
S31508003E480B600222204600F04FF8B0E7B2F864216A
S31508003E58002A95D001F07F0503FB050505F5AA7527
S31508003E68DEE7204603F0F2F908B10123DBE728600C
S31508003E78DAE70B7803704B784370CA788B7843EA8D
S31508003E88022343804A790B7943EA02238380CA7955
S31508003E988B7943EA0223C380704710B5802104460C
S31508003EA803F0B8F920460021BDE8104003F0B2B97E
S31508003EB830B588B105462B1A15F8014BDBB2002C2C
S31508003EC8F9D101335B0013800B7003234B7001385B
S31508003ED8022310F8012F02B930BDCA545A1CD2B2AF
S31508003EE802338C54DBB2F4E710B513460222C0F845
S31508003EF89422C0E906330A46002103F0C9F90020CE
S31508003F0810BD08B513460A46002103F0C1F900207A
S31508003F1808BD08B513460A46002103F0C7F900206C
S31508003F2808BD08B50423C0F8943200231A46194672
S31508003F3803F0AEF9002008BD08B50523C0F8943289
S31508003F4800231A46194603F0B1F9002008BD72B6CF
S31508003F58704762B670470000F0B58BB06846FEF742
S31508003F68ADFA2A4D029C00210E464FF4FA774FF413
S31508003F787A73B4FBF3F46B184A5D5B78D01800FBC8
S31508003F880770B4FBF0FC00FB1C4028B91FFA8CF636
S31508003F98701EB0F5806F08D302312429EBD1B521FC
S31508003FA81B4800F0B1FC00231A461A4C1A4921602E
S31508003FB8013A013B0025012712041B052046226108
S31508003FC8636125766576A576E77625776577C4E904
S31508003FD802556660FCF70CFE4CF6E0434FF6E072B5
S31508003FE8CDE900350423CDE9022369460E23204688
S31508003FF80993CDE90555079704950897FCF774FEC4
S315080040082046FCF7F5FE0BB0F0BD00BF2574000886
S31508004018E9730008D40400200064004030B589B06C
S3150800402840F2E17302930023CDE904330691024670
S3150800403801AB02A90A48FCF706FF78B900F0BEFAF0
S31508004048074C00F1320501992046FCF749FF28B1CB
S3150800405800F04BFD00F0B2FAA842F4D909B030BD19
S31508004068D404002010B588B00C46034601AA0021DE
S315080040780848FCF745FF58B9019A40F267639A421F
S3150800408804D1039B13B9059B2370012008B010BD02
S315080040980020FBE7D4040020FFF759BF10B500F04D
S315080040A8BFF9C8B1FCF710FAB0B100F0E5FCFCF7A7
S315080040B82BFD00F059FA00F0B5F9084B20F06040DE
S315080040C820F07F00986000F0ADF94468FFF741FFDB
S315080040D82346BDE81040184710BD00BF00ED00E0B4
S315080040E8F8B51446461A4FF6FF75013CA4B2AC4219
S315080040F800D1F8BD0B788B554F1C00F0F6FC3946F5
S31508004108F3E70000F8B50B4E054600240C2700F027
S31508004118ECFC07FB04F39A59AA4206D833445968B3
S315080041280A44AA4201D9187AF8BD01340A2CEED1F4
S31508004138FF20F9E74C7400082DE9F8430546FDF712
S3150800414825F8002405F104082F6858F8046004EBDC
S31508004158070900F0CAFC3246002349460220FDF743
S315080041685BF860B9E359B3420BD10434B4F5007F60
S31508004178EAD10124FDF71CF82046BDE8F883002497
S31508004188F8E70446F6E7000038B50E4B98420446A9
S315080041980D4607D00C4A914212D0FFF7CDFF10B949
S315080041A804460BE0094C23689D4207D020464FF485
S315080041B8007240F8045B2946FFF792FF204638BD8F
S315080041C81C46F0E70007002000800008FC040020D1
S315080041D82DE9F0419846036821F4FF760133044631
S315080041E80D46174626F0010606D140F8046B4FF42B
S315080041F800723146FFF774FF2368B34205D020469C
S315080042083146FFF7C1FF0446E8B123680435ED1ABD
S31508004218254406F50076B84400F067FC231DEB1A1A
S31508004228B3F5007F06D320463146FFF7ADFF0446AF
S3150800423848B1051D17F8013B05F8013B4745EBD181
S315080042480120BDE8F0810020FBE70000034A4FF093
S31508004258FF331360024A1360704700BFFC0400204E
S3150800426800070020124B70B51B1A16464A1E9A42BA
S3150800427804460D4619D8FFF745FFFF2815D0601ED6
S315080042882844FFF73FFFFF280FD024F4FF73094A95
S3150800429823F00103934221462B4632460CBF0648B3
S315080042A80648BDE87040FFF793BF002070BD00BF01
S315080042B8FFFF0F080080000800070020FC04002004
S315080042C870B51C4B4A1E1B1A9A4286B004460E46FF
S315080042D803D90024204606B070BDFFF713FF05462C
S315080042E8601E3044FFF70EFFFF2D0646F1D0FF2863
S315080042F8EFD00024012D0094ECD90B28EAD8854282
S31508004308E8D8012302220194CDE90432FCF73EFFDE
S3150800431800F0EBFB694601A80395FDF727F838B9BD
S315080043280135EBB29E42F3D20124FCF741FFD1E7EF
S315080043380024FAE7FFFF0F0807B50F4A1368013389
S3150800434817D0D2E901310B44D1680C480B441169DE
S315080043580B4451690B449169D2690B44134402AA68
S315080043685B4242F8043D0421FFF77CFF03B05DF881
S3150800437804FB0120FAE700BF00070020888100082F
S315080043880D4B0E4A1B68126813440D4A12681344EB
S315080043980C4A126813440C4A126813440B4A1268EA
S315080043A813440B4A126813440A4A1268D3420CBFCC
S315080043B801200020704700BF00800008048000081C
S315080043C8088000080C80000810800008148000087F
S315080043D818800008888100080A4808B50368013368
S315080043E805D109480368013306D1012008BDFFF73E
S315080043F8A3FE0028F5D1F9E7FFF79EFE003018BF9F
S315080044080120F3E700070020FC0400200048704755
S3150800441800800008FFF71ABFFFF724BFFFF750BF51
S31508004428FFF7AEBFFFF7F2BF08B5FFF785FF18B16C
S31508004438BDE80840FFF7D0BF08BD000038B5084CEE
S31508004448606000F0BBF800F10A0523681B0605D46E
S3150800445800F04BFB00F0B2F8A842F6D938BD00BF09
S315080044680044004010B50D4CE36823F4005388B0A7
S31508004478E3604FF461420023CDE9012301A90C2228
S315080044882046CDE90333CDE905230793FEF758F807
S31508004498E36843F40053E36008B010BD00440040E5
S315080044A8402970B506460C4603D97B21094800F011
S315080044B82BFA2046FFF7C2FF3546A4B2AB1B9BB2C0
S315080044C89C4200D870BD00F010FB15F8010BFFF7E9
S315080044D8B5FFF3E7C4740008F8B51E4D1E4A2C78D4
S315080044E80E46ACB913689B0602D400242046F8BDCC
S315080044F853681A4ADBB21370013B3F2BF5D800F014
S315080045085DF8174B1860174B1C7001232B70EDE7E5
S31508004518146814F0200414D0124C104923785768EC
S31508004528CA18013357700A78DBB29A422370DCD16D
S315080045380131FFF7D5FD00232B702378337001244A
S31508004548D4E700F03BF8064B1B6864339842CCD98D
S315080045582C70CBE7450900200044004004090020D8
S315080045684809002046090020024B00221A605A60B2
S315080045789A60704710E000E008B5FFF7F5FF054BAD
S31508004588054A5A60052100229A601960034B1A6089
S3150800459808BD00BF10E000E03F9002004C0900206B
S315080045A8044B1B68DB0341BF034A136801331360D6
S315080045B8704700BF10E000E04C09002008B5FFF777
S315080045C8EFFF014B186808BD4C09002008B5FFF72E
S315080045D8E7FF014B186808BD4C090020012838B5C3
S315080045E804460D4604D94FF4E0710E4800F08CF9DC
S315080045F80D49182060430B185C7C1A7C94420ED02F
S31508004608DA6815705A7C5C6801325A74DA680132BD
S31508004618A242DA6001D90A58DA60012000E00020CF
S3150800462838BD00BF0275000890090020012870B53A
S3150800463805460E4604D94FF4F1710D4800F064F9A1
S315080046480C4C18226A43A318587C80B199680978D3
S315080046583170597C58680139597499680131814211
S3150800466888BFA25899604FF0010088BF9A6070BD4C
S31508004678027500089009002038B51F4B1F4903F139
S3150800468818025A6140240022481C0A70C3E902002D
S31508004698186008191A4958600A601A491C82481C81
S315080046A8C3E908001C8598610819174CD8610125C3
S315080046B8DA629A7483F82A500D7020461349FFF770
S315080046C86FF813492046FFF79EF82846FBF710FFB0
S315080046D82046FFF7ABF8D4F8C402FDF79BFB00F0B9
S315080046E845F9B0F5FA6F05D24FF4FA60BDE83840D7
S315080046F800F036B938BD00BF90090020C40900206B
S31508004708C0090020050A0020480A00207400002075
S315080047181000002010B5064CD4F8C402FDF796FB25
S315080047282046FFF755F80020BDE81040FBF7E0BE25
S31508004738480A00203F292DE9F04107460C4603D9C7
S31508004748B921134800F0E0F8124D21462878FFF7FA
S3150800475845FF012803D0BD210D4800F0D5F8DFF83C
S3150800476830803E46A4B2F31B9BB2A34201D3BDE8F0
S31508004778F08100F0BAF916F8011B2878FFF72EFF22
S315080047880128F0D0C621404600F0BEF8EBE700BF86
S3150800479802750008C40900202DE9F8431E4B1F4E70
S315080047A81F4D8046D3F8C4020F46FDF77BF83478C8
S315080047B81C4B8CB929461878FFF738FF012803D00F
S315080047C800242046BDE8F8832B78013B3E2BF7D812
S315080047D8154B30701C70F4E7DFF84C90187899F888
S315080047E8001001312944FFF721FF01280446E7D1C3
S315080047F899F800302A780133DBB29A4289F80030F2
S31508004808DED1691C4046FFF76BFC0023337099F824
S3150800481800303B70D5E700BF480A0020580D002035
S31508004828180D0020050A0020590D00202DE9F3412E
S31508004838184E3478012C04D940F20221164800F0A3
S3150800484863F8164B182202FB0434647CFCB1402C2E
S31508004858DFF84480124F28BF402400250DF10701D0
S315080048683078FFF7E3FE012804D04FF4A3714046D9
S3150800487800F04AF89DF80730EB550135EBB29C4233
S31508004888ECD82346064A0748812102F001FD02B002
S31508004898BDE8F081C40900200275000890090020C7
S315080048A850090020480A00202DE9F041044602F084
S315080048B871FB214605461148114FDFF8488002F07A
S315080048C803FD2C4686B2631B9BB29E4209D802F0AA
S315080048D861FB4023024601210848BDE8F04102F081
S315080048E8E5BC14F8011B3878FFF778FE0128EAD0EA
S315080048F84FF4B471404600F007F8E4E7480A002088
S31508004908050A00200275000808B500F0EEF8FCE76D
S3150800491810B500F0E1F801281AD000F067F9B8B127
S315080049280C4C2378012B13D1FFF748FE0A4B0B4A88
S315080049381B681268134403F5FA73984208D30023D0
S31508004948237000F05BF918B9BDE81040FFF7A6BB5D
S3150800495810BD00BF600D00205C0D0020640D00200E
S31508004968014B1860704700BF5C0D0020014B1868A2
S31508004978704700BF5C0D002008B5044B1B78012B57
S3150800498803D1FFF71BFE024B186008BD600D002017
S31508004998640D002008B5044B01221A70FFF7ECFFD6
S315080049A8BDE80840FFF7B4BF600D002008B5FFF75B
S315080049B873FB00F098F8FFF7DFFDFFF72BFD00F013
S315080049C8FDF800F011F8BDE80840FFF7E3BF08B5A1
S315080049D800F08BF8FFF7E4FD00F008FA00F018F885
S315080049E8BDE80840FFF794BF10B5084C00F0D4FBA3
S315080049F8FFF7B2FA01232370FFF734FD002323706B
S31508004A08FFF73AFE0223237010BD00BF0D000020F1
S31508004A1807B517480DF10701FFF724FB012806D14A
S31508004A28144B9DF807101870114800F0D1FB0DF1CA
S31508004A3807010F48FFF750FD012807D10D4B9DF8D0
S31508004A4807100B4800221A7000F0C2FB0DF1070187
S31508004A580748FFF7A1FE012807D1064B9DF807105E
S31508004A68034802221A7000F0B3FB03B05DF804FB92
S31508004A78680D00200D000020FFF74CBE70B50D4CE0
S31508004A882378012B06460D4602D1C9B2FFF7C6FAA6
S31508004A9823781BB9E9B23046FFF702FD2378022BC3
S31508004AA803D1E9B23046FFF745FEBDE8704000F08D
S31508004AB887BB00BF0D000020044B1B78013BDBB207
S31508004AC8022B9ABF024AD05C402070470D0000208E
S31508004AD83E750008FFF7F0BF08B500F069FB00301F
S31508004AE818BF012008BDFBF7FDBCFBF7FEBC09286B
S31508004AF810B502D93730C0B210BD3030C4B202F092
S31508004B080BFC20442346427802F00302022A08BF17
S31508004B18A4F12003D8B2EFE738B5054600090C46D4
S31508004B28FFF7E5FF207005F00F00FFF7E0FF002309
S31508004B386070A370204638BDF8B5471E461C002588
S31508004B4817F8014F02F0E8FB20442346427802F0A2
S31508004B580302022A08BFA4F12003DBB2A3F130023C
S31508004B68D2B2162A0FD8A3F13A0106290BD9092A6F
S31508004B7884BF373BDAB202EB0513BE4203F0FF05E2
S31508004B88DED12846F8BD0025FBE7000003460246A5
S31508004B9809480A210130B2FBF1F2002AFAD102705B
S31508004BA80A21B3FBF1F201FB1233303300F8013D59
S31508004BB81346002AF5D170479013002008B5074B0D
S31508004BC80749084800221A7001F0FEFC28B1772127
S31508004BD80548BDE80840FFF797BE08BD081200203B
S31508004BE841750008B00D002044750008024B187876
S31508004BF8B0FA80F0400970470812002010B5FFF790
S31508004C086BFF012801D1002010BD054C2378002B25
S31508004C18F9D1FBF79DFC0128F5D12070F4E700BF10
S31508004C280812002038B50546047802F075FB2044BA
S31508004C382346427802F00302022A08BFA4F1200399
S31508004C48532B0CD102F068FB6B781844427852074C
S31508004C5805D5312B05D0322B05D0332B05D00320AB
S31508004C6838BD0020FCE70120FAE70220F8E770B50E
S31508004C7805460230FFF760FF0435044686B2284623
S31508004C88FFF75AFF013EB6B20444012EE4B205F115
S31508004C980205F4D82846FFF74FFFE443E4B2231A7F
S31508004CA85842584170BD00002DE9F04104461746A0
S31508004CB80E4601B120B940F263214B48FFF724FE9E
S31508004CC82046FFF7AFFF032805460AD02046FFF718
S31508004CD8CEFF002800F08480012D27D003D3022DAB
S31508004CE84DD000251AE0A01CFFF726FF0546201D13
S31508004CF8FFF722FF00023060A01DFFF71DFF33688B
S31508004D08033D184430602DB247B1083400239EB2DB
S31508004D18AE4204EB430003F1010802DB2846BDE86E
S31508004D28F081FFF709FF4346B855F0E7A01CFFF7DF
S31508004D3803FF0546201DFFF7FFFE00043060A01D8F
S31508004D48FFF7FAFE336803EB0020306004F1080029
S31508004D58FFF7F2FE3368043D184430602DB2002F81
S31508004D68DCD00A3400239EB2AE4204EB430003F1BA
S31508004D780108D3DAFFF7E0FE4346B855F3E7A01C67
S31508004D88FFF7DAFE0546201DFFF7D6FE0006306057
S31508004D98A01DFFF7D1FE336803EB0040306004F12D
S31508004DA80800FFF7C9FE336803EB0020306004F1FA
S31508004DB80A00FFF7C1FE3368053D184430602DB276
S31508004DC8002FABD00C3400239EB2AE4204EB43004E
S31508004DD803F10108A2DAFFF7AFFE4346B855F3E731
S31508004DE84FF0FF359AE700BF447500082DE9F84FDC
S31508004DF8BE4D2E78A84666B3012E2CD1FFF70AFBBE
S31508004E08FBF7C6FBBA48FBF701FCBA48FBF7FEFBFB
S31508004E18FBF7BAFB32460146B74801F0FDFB0446E4
S31508004E2848B10023B5482B70FBF7F0FB3046BDE8C0
S31508004E38F84FFBF7E1BBB248FBF7E8FBB148FBF7CD
S31508004E48E5FBB148FBF7E2FBB04BC3E90044022394
S31508004E582B70BDE8F88F022E40F0C980DFF8D0A283
S31508004E68AB4C0AF50C724FF48071204601F076FFB8
S31508004E789AF841B25746A146BBF1000F0DD0002358
S31508004E889E482B70FBF7C2FB3046FBF7B5FB0AF5C5
S31508004E980C70BDE8F84F01F03BBEC8B15A4604F598
S31508004EA8C0712046FFF700FF431C064606D1934803
S31508004EB885F800B0FBF7AAFB0320E6E7002807DD1C
S31508004EC8924BD4F880015A681C46AAB918605E60E5
S31508004ED8D7F84422D7F83C329A42BAD100218648F4
S31508004EE801F023FE00284DD00023844888F80030B6
S31508004EF8FBF78CFB042036E019681144814201D17E
S31508004F081644E4E77E48FBF781FB8248FBF77EFBFD
S31508004F186068FFF73BFE8048FBF778FB7F48FBF79E
S31508004F2875FB7D49E078FFF7F7FD7D49A078FFF71F
S31508004F38F3FD7C496078FFF7EFFD7B492078FFF79A
S31508004F48EBFD7548FBF762FB7848FBF75FFBD4E98E
S31508004F580001FFF763FA50B90023684888F800305B
S31508004F68FBF754FB0520FBF747FB634891E76448C2
S31508004F78FBF74CFB6448FBF749FBD9F88031C4E9D1
S31508004F880036A5E7614C636853B35D48FBF73EFBFB
S31508004F986048FBF73BFB6068FFF7F8FD5E48FBF7E0
S31508004FA835FB5E48FBF732FB5B49E078FFF7B4FD53
S31508004FB85B49A078FFF7B0FD5A496078FFF7ACFD62
S31508004FC859492078FFF7A8FD5348FBF71FFB5748B0
S31508004FD8FBF71CFBD4E90001FFF720FA0028BBD031
S31508004FE84748FBF713FB032388F8003031E7032EFD
S31508004FF87FF42FAF4E4F464C07F50C724FF480716D
S31508005008204601F0ABFE97F841B2BA46BBF1000F4D
S315080050180AD0002347482B70FBF7F8FA0220FBF75B
S31508005028EBFA07F50C7034E700284AD004F58072C5
S3150800503804F5C0712046FFF737FEB0F1FF3F8146F9
S3150800504806D13D4885F800B0FBF7E0FA3046E6E7B2
S31508005058002836DD3948FBF7D9FA4846FFF796FDA2
S315080050682D48FBF7D3FA3648FBF7D0FA2A4994F8BD
S315080050788301FFF751FD2A4994F88201FFF74CFD91
S31508005088284994F88101FFF747FD274994F88001D4
S31508005098FFF742FD2048FBF7B9FA2448FBF7B6FAAA
S315080050A804F580724946D4F88001FFF7B5F928B99E
S315080050B828701248FBF7AAFA0620B0E71048FBF74B
S315080050C8A5FADAF84422DAF83C329A427FF4C1AEF5
S315080050D81C48FBF79BFAFFF7A7F9A8BB88F8000056
S315080050E80648FBF793FA07203DE700BF0812002099
S315080050F87275000895750008E00F00206F7600089D
S31508005108BA750008BF750008E3750008A80D0020E1
S315080051180C12002013760008901300201C7600084D
S31508005128921300209413002096130020B6750008E1
S31508005138B00D002035760008567600087776000800
S31508005148847600089B7600080A48FBF75FFA0A483F
S31508005158FBF75CFA094801F0DBFC0948FBF756FA45
S31508005168002388F80030FBF727FABDE8F84FFEF762
S3150800517895BF00BFBA750008B7760008E00F00208B
S31508005188CF760008034BFE22DA7002221871A3F8BC
S3150800519844207047D0130020044B00229A6483F8F1
S315080051A84320A3F844201A809A707047D013002029
S315080051B8024B1878003018BF01207047D01300201A
S315080051C8024B002283F84320704700BFD013002003
S315080051D8F8B50678804CFF2E054633D1FFF706FD4D
S315080051E818B91020FFF7CEFF17E010230125237101
S315080051F8002363712580E670FFF75EFCA071FFF750
S3150800520869FCE071FFF766FC0823000A20726572DC
S31508005218A572A4F84430FFF7FDF894F84330012B3B
S3150800522802D11020FFF7AEFFB4F94410002940F365
S31508005238D280012384F8433089B26848BDE8F8402B
S31508005248FFF71CBC2778012F40F0C580F32E56D0EF
S315080052581FD8CF2E00F0BC8007D8C92E00F0818051
S31508005268CC2E00F087802020BCE7D12E00F0A9803C
S31508005278C0F08A80D22EF6D10025FF23E370257167
S315080052886571FFF719FCE571A07125726572072328
S3150800529829E0FA2E4AD00BD8F52E11D026D3F62EA9
S315080052A8E1D1FF23E3704368A364A4F84470B4E724
S315080052B8FD2E47D0FE2E4FD0FC2ED4D1002091E7E4
S315080052C8FFF7FAFB6A78904201D822208AE7A16C90
S315080052D8201DFEF705FFFF23E3706A78A36C1344C5
S315080052E8A3646B780133A4F8443096E7FFF7E4FB28
S315080052F86B788342E9D26968A1646A78E8E7FF238C
S31508005308E370A66C476800253744BE4207D10123D7
S31508005318A3800023C4F80750A3710823E3E716F807
S31508005328013B1D44EDB2FFF7E0FBEEE7FF23E37010
S315080053382B4BA364002323716371A3710723C4F855
S315080053480730EAE7FF23E370627862710023237166
S31508005358E38023720623C6E700232380FF23E3702E
S31508005368A3E7A66CFFF7A8FB6A1C411E3046FFF7A1
S3150800537853F808B9312035E7FF23E370FFF79CFB9C
S31508005388A36C013803448FE7FFF796FB6B7801385F
S3150800539898429ADDFF23E370A4F84470697829B91E
S315080053A8FFF742F800287FF438AFE3E7AA1CA06C99
S315080053B8FFF732F80028DDD06A78A36C1344A36493
S315080053C82BE74168A06CFFF729F80028C6D1D1E772
S315080053D8FEF764FEC2E7F8BDD0130020D3130020F9
S315080053E8F876000842884378007843EA022340EAB8
S315080053F80320704743690239023B8B4283BF4389BE
S31508005408806A01FB030000207047024600F10B0181
S315080054180020C30143EA500312F8010B50FA83F33C
S315080054288A42D8B2F5D17047026810B552B111460A
S315080054380B4611F8014B1F2C0CD93A2CF8D1511CE4
S315080054488B4202D04FF0FF3005E01278302AF9D1A6
S3150800545801330360002010BD38B50D46044618B957
S3150800546800232B60092038BD0368002BF8D01A786A
S31508005478002AF5D0D98882889142F1D15878FDF763
S31508005488F7FF10F00100EBD123682B60EBE7013832
S315080054980A4411F8013B00F8013F9142F9D17047D7
S315080054A8CA7E8B7E032843EA022301BF487D0A7D0C
S315080054B842EA002243EA024318467047C2F3072322
S315080054C88A76CB760378032B01BF120C0A75120A63
S315080054D84A757047F8B5C56A00F1300704460123CE
S315080054E82A4639464078FEF70FF8A0B9236AA26912
S315080054F8E070EB1A934201D30020F8BDA678012E76
S31508005508FAD9A36960781D442A4601233946FDF766
S31508005518FBFF013EF3E70120EFE7C3780BB1FFF77E
S31508005528D9BF18467047C36A8B4270B506460D46FA
S3150800553812D0FFF7F2FF044660B92A46012306F19E
S3150800554830017078FDF79EFF00281CBF4FF0FF3525
S315080055580124F562204670BD0024FBE738B5002310
S31508005568C3704FF0FF33C3620446FFF7DCFF0146FA
S31508005578E8B994F82F2294F82E3243EA02234AF619
S315080055885522934215D104F16600FFF72BFF0B4D00
S3150800559820F07F40A8420ED004F18200FFF722FFD0
S315080055A820F07F40A84214BF0220002038BD0420FE
S315080055B8FCE70320FAE70846F8E700BF4641540027
S315080055C82DE9F043002385B00B600F461546FFF713
S315080055D82BFF061EC0F22E81994B53F82640002C45
S315080055E800F02A813C60237805F0FE0573B16078DF
S315080055F8FDF73EFFC10709D4002D00F0F68010F02C
S31508005608040000D00A2005B0BDE8F0830023F0B2F4
S3150800561823706070FDF7E2FDC20700F10F810DB136
S315080056284307EFD400212046FFF798FF022840F0E9
S31508005638E78004F5FB75002115F8040C10B1284617
S31508005648FFF7D0FE4DF821000131042905F11005B0
S31508005658F2D100265DF82650002D00F0C8802946AC
S315080056682046FFF77BFF012800F2C28094F83C2009
S3150800567894F83B3043EA0223B3F5007F40F0C48030
S3150800568894F8473094F8466056EA032604D104F19C
S315080056985400FFF7A7FE064694F84090A66109F15C
S315080056A8FF33012B84F8029000F2AE8094F83D701F
S315080056B8BBB26381002B00F0A7807B1E3B4240F0FB
S315080056C8A38094F8423094F8418048EA032818F0F1
S315080056D80F0FA4F8088040F0978094F8441094F8BF
S315080056E8430050EA012003D104F15000FFF77AFE7F
S315080056F894F83F2094F83E3053EA022300F0848059
S3150800570806FB09FC03EB1812624490427CD3811A03
S31508005718B1FBF7F1002977D040F6F577B94294BF7F
S31508005728012702274FF6F570814288BF03272B44C5
S3150800573802312A44032F6161E5612362A26267D1B7
S3150800574894F85B2094F85A3053EA02235CD1B8F1EE
S31508005758000F59D104F15C00FFF744FE6062890026
S3150800576801F2FF11B6EB512F4ED34FF0FF33C4E9C0
S315080057780333032F4FF0800323712FD194F8612048
S3150800578894F8603043EA0223012B27D1691C204686
S31508005798FFF7C9FE10BB94F82F2294F82E32207111
S315080057A843EA02234AF65522934217D104F13000F8
S315080057B8FFF718FE234B984210D104F50570FFF73A
S315080057C811FE214B984209D104F50670FFF70AFE27
S315080057D8206104F50770FFF705FEE0601B4A27708D
S315080057E8138801339BB21380E38000200BE703205C
S315080057F80136042E7FF42EAF042805D1012002E7CE
S315080058080428FBD0012801D90D20FCE600252DE740
S31508005818B8F1000FF8D0022F4FEA410018BF401818
S31508005828634418BF01F0010163620CBF014601EB2E
S31508005838500195E70B20E6E60C20E4E60320E2E6AD
S315080058481C140020525261417272416120140020D2
S315080058580129F8B506460C4652D9436999424FD2EA
S315080058680378022B29D0032B39D0012B48D101EB19
S315080058785105016A01EB5521FFF755FE10B14FF0A6
S31508005888FF30F8BD6F1C316AC5F30805354401EBCE
S315080058985721304695F83050FFF745FE0028EED1D7
S315080058A8C7F308073E44E30796F8300045EA0020A0
S315080058B84CBF0009C0F30B00E3E7016A01EB1421AA
S315080058C8FFF731FE0028DAD1640004F4FF74344483
S315080058D894F8313094F8300040EA0320D1E7016A99
S315080058E801EBD411FFF71FFE0028C8D1A00000F469
S315080058F8FE7030303044FFF775FD20F07040C0E781
S315080059080120BEE7B1F5001FF8B506460D4601D3D6
S315080059180220F8BDCA06FBD1826804683161C2B99B
S315080059282378022B01D9636AA3B92389B3EB551FD8
S31508005938EED9636AB361B3697261002BE8D003EBE9
S3150800594855233034C5F308052C44B361F4610020A7
S31508005958DFE7134667891A467F02BD42114604D215
S315080059682046FFF747FDB061E5E73068FFF770FFA7
S31508005978431C024606D00128CAD963698342C7D997
S31508005988ED1BEAE70120C4E701292DE9F04106469F
S315080059980C46154678D943698B4275D90378022B84
S315080059A83FD0032B50D0012B6ED101EB5107016A6A
S315080059B801EB5721FFF7B7FD014638BB07F1010888
S315080059C8C7F30807374414F001041FBF97F83030A7
S315080059D803F00F022B0103F0F00314BF1343EBB2D5
S315080059E887F83030316A012301EB5821F3703046C5
S315080059F8FFF799FD014648B9C8F30803334444B18B
S31508005A08C5F3071583F830500123F3700846BDE837
S31508005A18F08193F83020C5F3032522F00F021543C9
S31508005A28F0E7016A01EB1421FFF77DFD014600281E
S31508005A38ECD1640004F4FF74344484F83050C5F398
S31508005A48072584F83150DFE7016A01EBD411FFF71F
S31508005A586AFD01460028D9D1A40004F4FE7404F1AD
S31508005A68300737443846FFF7BDFC25F0704500F087
S31508005A78704028433444030A84F830007B70030CCA
S31508005A88000EBB70F870BFE70221BFE72DE9F041A9
S31508005A98804605680F4671B9EE68F6B16B69B34278
S31508005AA898BF012634466B690134A34218D8012EDB
S31508005AB815D8002409E02846FFF7CAFE0128044637
S31508005AC837D9431C04D14FF0FF342046BDE8F0818E
S31508005AD86B698342F9D83E46E4E70126E2E70224E1
S31508005AE82146D8F80000FFF7B3FE30B1012820D0C8
S31508005AF80130E8D0B442D6D1DBE74FF0FF32214671
S31508005B082846FFF741FF90B957B9D5E90432023A52
S31508005B189342EC600FD32B7943F001032B71D4E73A
S31508005B28224639462846FFF72FFF0028EDD00128D8
S31508005B38C9D00124C9E7013B2B61ECE7F8B50D4646
S31508005B48012D074611462BD904686369AB4227D944
S31508005B582AB14FF0FF322046FFF716FF30B929461B
S31508005B683868FFF775FE064608B90020F8BD01280B
S31508005B7816D0411C16D0002229462046FFF704FFF6
S31508005B880028F3D123695A1C05D0013323612379E8
S31508005B9843F0010323716369B3423546DFD8E4E766
S31508005BA80220E3E70120E1E7436A01332DE9F041E2
S31508005BB806460C460BD0D0F8288001F116070025B2
S31508005BC838F81500002851D125440023AB75F1692A
S31508005BD8A07D01F10B0E0D4600232E2615F8012B84
S31508005BE8202A24D0052AA5EB010C08BFE522BCF11A
S31508005BF8090F04D1E71800B9BE757E720133E71894
S31508005C087A7298B9A2F14108B8F1190F0DD8BCF102
S31508005C18090F91F80C8034BF4FF0080C4FF0100CA0
S31508005C2818EA0C0F1CBF2032D2B2BA750133AE453A
S31508005C38D4D128B9E21890750A7B002A08BF002330
S31508005C48234400225A72CB7A237201F11C00FFF70B
S31508005C58C9FB20604A7E0B7E43EA0223A380CA7DDD
S31508005C688B7D43EA0223E380BDE8F081002101F039
S31508005C78BDF828B1FF2D03D0013507F8010B9FE7BA
S31508005C880025A1E783692DE9F04705468946A3B1AA
S31508005C9807692037B7F5001F0FD2C7F30808046845
S31508005CA8B8F1000F51D141690133836139B92389A4
S31508005CB8B3EB571F49D80023AB6104200BE063896F
S31508005CC8013B13EA572340D12046FFF7C1FD0128B7
S31508005CD8064602D80220BDE8F087421C01D10120F9
S31508005CE8F9E7636983422AD8B9F1000FE3D06969ED
S31508005CF82846FFF7CBFE064600283AD00128E9D001
S31508005D08431CECD02046FFF708FC0028E7D104F12D
S31508005D18300304F50C7203F8010B9342FBD13146A4
S31508005D282046FFF767FB4FF00009E0624FF0010ACB
S31508005D386389994510D3E36AA3EB0903E3626E61A5
S31508005D4831462046FFF756FBA86108F13008444457
S31508005D582F61EC610020BEE784F803A02046FFF710
S31508005D68B9FB0028BBD1E36A013309F10109E362EB
S31508005D78DEE70720AFE7416A4B1C2DE9F0410446E8
S31508005D880568066918D1E5274FF00108A16928466C
S31508005D98FFF7C9FB60B9E3691F7085F803802369B3
S31508005DA8B3420DD201462046FFF76CFF0028EDD016
S31508005DB8042808BF022003E0FFF7A4FD0028E2D064
S31508005DC8BDE8F0812DE9F04F85B0036801930021FD
S31508005DD80546FFF797FD8046002840F098804FF063
S31508005DE8FF334FF0FF0A6B625646A9690198FFF719
S31508005DF89AFB8046002840F08A80EC692778002FAD
S31508005E0800F08980E27AE52F02F03F03AB7103D0F0
S31508005E18100705D50F2B05D04FF0FF336B6256E0F8
S31508005E280F2B5BD1D5F828B0BBF1000F45D0790602
S31508005E384BD52A6994F80DA06A6207F0BF07627BFA
S31508005E48524544D1E27EA67E46EA022636B2002E9E
S31508005E583DD194F8008008F03F0808F1FF324FF06A
S31508005E680D0808FB02F801212C4BF25CA01814F85F
S31508005E780290407849EA002959B3B8F1FE0F26D8A6
S31508005E88484600F0D1FF08F1010203903BF81800D4
S31508005E98029200F0C9FF0399814218D1029A49462D
S31508005EA8904601360D2EDFD12278520603D511B158
S31508005EB83BF818305BB9013FFEB200212846FFF7C8
S31508005EC8E1FE8046002890D021E0BE42B7D0FF26E2
S31508005ED8F3E74FF6FF739945E3D0F8E726B9204666
S31508005EE8FFF793FA504512D02A6AD37ADB0793D478
S31508005EF804F10B0114F8013B12F8010B8C42A3EBD1
S31508005F08000302D0002BF5D086E7002B84D1404643
S31508005F1805B0BDE8F08F4FF00408F8E78077000869
S31508005F282DE9F84FFF250668464F81462C464FF05F
S31508005F38040A4FF6FF78D9F8181019B9BAF1000FFC
S31508005F4873D062E03046FFF7EEFA824600285CD145
S31508005F58D9F81C000378002B71D0C27AE52B02F019
S31508005F683F0289F8062056D02E2B54D022F020015D
S31508005F78082950D00F2A53D15A064AD503F0BF0428
S31508005F88D9F81030457BC9F82430437BAB4242D157
S31508005F98C27E837E43EA02231BB2002B3BD10278DA
S31508005FA8D9F8281002F03F02013A4FF00D0C0CFB05
S31508005FB802FC4FF0010E13F807A000EB0A0292F84C
S31508005FC801B010F80A2042EA0B22BEF1000F24D0CD
S31508005FD8BCF1FE0F1FD821F81C2096460CF1010CBF
S31508005FE801330D2BE7D103785B0605D5BCF1FE0F07
S31508005FF811D8002321F81C30013CE4B20021484698
S31508006008FFF740FE8246002895D00023C9F81830C5
S315080060180DE0A342B9D0FF24F0E74245E0D0FAE7FD
S3150800602844B9FFF7F2F9A84204D14FF0000A5046DE
S31508006038BDE8F88F4FF0FF33C9F82430F7E74FF07B
S31508006048040AE2E7807700082DE9F74F036800930A
S3150800605807468A4611F8013B2F2BFAD05C2BF8D055
S315080060680021B9609AF800301F2B00F2AC803B6A11
S3150800607880223846DA7203B0BDE8F04FFFF742BC13
S315080060885C2800F0B080B4F5807F0BD0012100F0C1
S31508006098ADFE38B17F2807D8804911F8012F1AB103
S315080060A89042FAD106204DE025F8020F264691E0DF
S315080060B832F8021D202902D02E2940F0A680013E7A
S315080060C8A0E00131B2E0C14505D296424AD1B8F1FD
S315080060D80B0F3FD102E0B8F10B0F36D144F0030499
S315080060E84FF00B083B6A1A78E52A04BF05221A708E
S315080060F8B8F1080F04BFAD00EDB205F00C030C2B80
S3150800610803D005F00302032A01D144F00204A107CB
S3150800611809D405F00305012D08BF44F01004042B23
S3150800612808BF44F008043B6A3846DC72FFF74AFEA3
S315080061383B6ADB7A002837D0042803D113F0040F0A
S3150800614808BF052003B0BDE8F08F964202D044F098
S315080061580304C7D3AD00EDB232464FF00B084FF033
S31508006168080989E07F280CD90021019200F03EFE33
S3150800617844F00204019A58B1494B184410F8800CA7
S3150800618830B1484B13F8011F002979D08142F9D15B
S3150800619844F003045F20396A01F8090009F1010986
S315080061A86AE045F00205F6E75A07CBD4BB79DB0661
S315080061B864D53969009BC1F3080130311878194448
S315080061C8FFF76EF9B860D7F828B00AF1FF38ABF1CF
S315080061D80205002618F8010F1F2806F1010402D93E
S315080061E82F287FF44DAF544422782F2AA24604F16B
S315080061F80104F9D05C2AF7D01F288CBF0024042490
S315080062080BEB4602002E7FF453AF00210BEB460238
S315080062182BF81610002E3FF445AF396A202501F1F0
S315080062280B0001F8015B8842FBD100213BF81100FD
S3150800623820283FF446AF2E283FF443AF09B144F06F
S31508006248030432F8020D2E2801D0013EF9D14FF089
S3150800625800094FF008084D463BF811004A1C00286B
S315080062683FF440AF202805D02E287FF42CAF96425D
S315080062783FF42DAF44F003041146EDE7052061E726
S31508006288A0F1410119298CD9A0F1610119299EBFEC
S31508006298203845F0010580B27DE700BF8C770008F5
S315080062A8007700089577000838B50446FFF735F9EA
S315080062B8002851D12378032B46D12379012B43D1C2
S315080062C804F1300104F50C720B46054603F8015B28
S315080062D89342FBD1552384F82E32AA2384F82F3209
S315080062E8522384F8303084F83130612384F8323008
S315080062F884F81732236984F81832412284F833203F
S3150800630884F816221A0A84F819221A0C1B0E84F81D
S315080063181B32E36884F81A221A0A84F81D221A0C12
S3150800632884F81E22E26984F81C3272201B0E013298
S3150800633884F8140284F8150284F81F32E2620123ED
S315080063486078FDF7E1F82571002211466078FDF7B7
S315080063583BF9003018BF012038BD00002DE9F04F81
S31508006368066AF47A14F0A00487B0054640F08480DB
S31508006378D0F8288038F81490B9F1000F5CD10C22AF
S3150800638831460DEB02002F68FFF781F89DF81730A4
S31508006398DB077BD586F80B90C5F82890DFF820929E
S315080063A84FF0010A0B2203A93046FFF770F8BAF135
S315080063B8050F52D9A8F10200534630F8022F002AD1
S315080063C83CD1072203F00F0000F13001392988BFB4
S315080063D800F13701013A01A810441B094170F1D1AF
S315080063E806A911447E2001F8140C934204D0F15CE6
S315080063F8202903F1010032D13344072A9BBF06A995
S315080064088918202111F8141C03F8011BA3EB0601AF
S3150800641898BF01320729F0D92846FFF7D3FC8346E7
S3150800642868BB0AF1010ABAF1640FBBD14FF0070B32
S31508006438584607B0BDE8F08F01349BE7102102F0F3
S31508006448010C0CEB430313F4803F18BF83EA0903D6
S3150800645801394FEA5202F2D1AFE75346B1E703468C
S31508006468C3E7064601212846FFF70CFC834618B3FE
S31508006478BBF1040FDAD0DBE74FF0060BD8E70428A0
S31508006488D6D19DF81730F372C5F828809DF81730CD
S31508006498D5F800809B0748BF0C344FF00001284602
S315080064A849BF0D230124B4FBF3F40134FFF72AFA94
S315080064B883460028DCD10646A9694046FFF733F823
S315080064C883460028D4D1EB691B78E52B01D0002B2D
S315080064D8C7D10136B442C5D1013C53D029692846EB
S315080064E8A1EB4411FFF70EFA83460028A0D1286AC3
S315080064F8DFF8D080FEF789FF4FF6FF790646A969C7
S315080065083846FFF710F88346002891D1EB69D5F885
S3150800651828E05E730F22E1B24FF00D0CDA724A1EBC
S315080065280CFB02F218739876D876844648451CF808
S3150800653808A018BF3EF8120003F80A0003EB0A0B76
S315080065480CF1010C18BF01324FEA102A002808BFBF
S315080065584846BCF10D0F8BF801A0E7D1484502D093
S315080065683EF812200AB941F0400119700123FB7060
S3150800657800212846FFF786FB834600287FF458AF94
S31508006588013CBCD1A9693846FEF7CDFF83460028E9
S315080065987FF44EAFEB69014603F1200203F8011BAD
S315080065A89342FBD10B22D5E90701FEF770FFD5E91F
S315080065B80723DB7A03F0180313730123FB7037E705
S315080065C821100100807700081FB5CDE9001004A83E
S315080065D8144640F8041DFEF727FF011E15DB0D4B70
S315080065E853F8210008B100220270019808B1002268
S315080065F8027043F8210030B1012C08D1002201A904
S315080066086846FEF7DDFF04B010BD0B20FBE7002047
S31508006618F9E700BF1C1400202DE9F04393B015468E
S3150800662801910446002800F09580002302F01F0611
S315080066380360324603A901A8FEF7C2FF002857D10E
S31508006648039B079304AB0F930199454B119307A82E
S31508006658FFF7FAFC28B90F9B93F90B30002BB8BF44
S31508006668062015F01C0F4FD0002844D004283FD127
S3150800667807A8FFF773FE00283AD146F0080635073B
S315080066884CD50E9BDDF80C8000256121482219742B
S315080066985A749D73DD730E9B19765A769D75DD754A
S315080066A80E9B2022DA72DDF8389098F800004946E1
S315080066B8FEF7F6FE2A4607464046FEF7FFFE0E9BFD
S315080066C81D775D779D77DD77039B0122DA702FB3F7
S315080066D82A46394607A8D3F82C80FFF72FFA38B97F
S315080066E841460398FEF71FFF039B013FDF60A8B1E9
S315080066F813B0BDE8F0839DF8223013F0110F2DD1A1
S315080067086F07BCD50820F3E70028F1D19DF8223099
S31508006718D80621D4A90701D5DA071FD4039D0E9FE9
S315080067283307EB6A236267622878394648BF46F01A
S315080067382006FEF7B5FEA06007F11C00FEF752FE1C
S31508006748E060002060742674EB886061E06125606B
S31508006758A380CDE70920CBE70420C9E70720C7E7C8
S31508006768221400202DE9F04F9B4685B00023894660
S31508006778CBF8003003A904461546FEF76DFE064613
S3150800678800BB667CF6B9237CD80740F18F80E3689E
S315080067986769DF1BAF4204F1280328BF2F46009319
S315080067A887B16269C2F30803002B70D1039B5B8922
S315080067B8013B13EA522315D142B9A06801280CD81F
S315080067C802266674304605B0BDE8F08FA1692068D0
S315080067D80193FFF73DF8019BF0E7411C01D101261B
S315080067E8EFE7A061DDF80CA0A16901935046FEF712
S315080067F801FE0028E4D0019B7D0A03EB000829D096
S31508006808BAF80A209AF801005919914288BFD51A88
S315080068182B4642464946FCF735FE0028DFD1237C3D
S315080068285A060BD5E069A0EB0800A84206D24FF431
S315080068380072009909EB4020FEF729FE6D0263698C
S315080068482B446361DBF800302B44A944CBF80030AD
S315080068587F1BA5E7E269424517D0237C5B060BD563
S31508006868012300999AF80100FCF74EFE0028B6D1D4
S31508006878237C23F040032374039800994078012366
S315080068884246FCF7FFFD0028A9D1C4F81C806169B7
S31508006898C1F30801C1F50075BD4228BF3D46283138
S315080068A82A4621444846FEF7F2FDC8E7072689E73F
S315080068B82DE9F04F9B4685B000238946CBF8003072
S315080068C803A904461746FEF7C7FD0646002840F002
S315080068D88880667C002E40F08480237C990740F1E6
S315080068E8AA806369FB4200D3DF4304F128030193B6
S315080068F85CE0A1696CE0012802D10226667470E0A2
S31508006908421C01D10126F9E7A368A06103B9A06072
S31508006918237C5B060CD50398E26901994078012324
S31508006928FCF7F2FD0028EDD1237C23F040032374FD
S31508006938DDF80CA0A1695046FEF75CFD0028DCD0FE
S31508006948009B7D0A03EB00084FD0009ABAF80A3074
S315080069589AF801002A449A4284BF009A9D1A2B463F
S3150800696842464946FCF7D0FD0028CBD1E169A1EBA0
S315080069780801A9420AD24FF4007209EB412101988D
S31508006988FEF785FD237C23F0400323746D026369B3
S31508006998E2682B4463619A422CBFE260E360DBF845
S315080069A800302B44A944CBF800307F1BAFB163698C
S315080069B8C3F3080262BB039A5289013A12EA5322C0
S315080069C80092A5D1002B94D1A068002893D101463E
S315080069D82046FFF75BF800288DD1237C43F0200377
S315080069E82374304605B0BDE8F08FE36943450DD0FA
S315080069F8E26863699A4209D90123424601999AF8D5
S31508006A080100FCF73FFD00287FF47CAFC4F81C8022
S31508006A186069C0F30800C0F50075BD4228BF3D4649
S31508006A2828302A4649462044FEF731FD237C43F0A0
S31508006A3840032374ABE70726D3E70A2973B5044648
S31508006A480E4602D10D21FFF7F8FF6368002B14DB09
S31508006A585D1C23443C2D1E730BDD01AB2A4604F14D
S31508006A680C012068FFF724FF019B5D1B18BF4FF038
S31508006A78FF35A36865600133A36002B070BD73B5BE
S31508006A8801A90546FEF7E8FC064600283BD12B7CFB
S31508006A989A0638D55B060CD50198EA694078012329
S31508006AA805F12801FCF730FD80BB2B7C23F0400359
S31508006AB82B74296A0198FEF736FD064618BB6C6AD8
S31508006AC8E37A43F02003E372AA6828682146FEF7AA
S31508006AD8F5FCEB6823771A0A62771A0C1B0EE3771C
S31508006AE8612323760198A675482363760123E675FC
S31508006AF8A674E674A277C370FFF7D6FB2B7C23F03F
S31508006B08200306462B74304602B070BD0126FAE704
S31508006B1813B50446FFF7B3FF28B901A92046FEF7BF
S31508006B289BFC00B9206002B010BDF7B50D4601A957
S31508006B380446FEF791FC0646002859D1667C002EC5
S31508006B4856D1E368AB4204D2227C12F0020F08BF82
S31508006B581D460022636962614DB96369E26893421A
S31508006B6881BFE360237C43F02003237440E0019A45
S31508006B7857897F02002B31D0013B6A1EB3FBF7F118
S31508006B88B2FBF7F28A4229D37A421340A1696361B4
S31508006B98ED1A002951D100256369C3F30803002BB0
S31508006BA8DBD0E269AA42D8D0237C5B0604F1280721
S31508006BB80AD50198012339464078FCF7A5FCE0B9BF
S31508006BC8237C23F040032374019801232A46394677
S31508006BD84078FCF757FC80B9E561BEE7A16879B942
S31508006BE82046FEF753FF0128014604D1022666749B
S31508006BF8304603B0F0BD431C01D10126F7E7A06073
S31508006C08A161C6E7237C980706D52046FEF73EFF0E
S31508006C18014628B93D4612E02068FEF719FE0146E6
S31508006C284A1CEAD00129E1D9019B5B698B42DDD967
S31508006C386369A1613B446361ED1BBD42E2D86369A0
S31508006C482B446361C5F30803002BA4D00198FEF70B
S31508006C58D1FB0028CAD000EB55259DE730B591B081
S31508006C680D460190002205A901A8FEF7A9FC0446CD
S31508006C78B0B902AB0D9301990C4B0F9305A8FFF712
S31508006C88E3F9044660B90D9B93F90B30002B0ADB30
S31508006C9835B10B9BA8751BB1294605A8FEF784FFD5
S31508006CA8204611B030BD0624FAE700BF221400209A
S31508006CB8F0B59DB00222019002A901A8FEF780FC52
S31508006CC8029B0693044698B903AB0E930199224B87
S31508006CD8109306A8FFF7B8F9044648B90E9B93F926
S31508006CE80B30002B36DB9DF81E70FA0703D50724F0
S31508006CF820461DB0F0BD029E0D993078FEF7D0FBF0
S31508006D08FB0605460BD406A8FFF735F804460028FF
S31508006D18EED1B5B90298FFF7C7FA0446E8E7139023
S31508006D28214611A81196FEF7EDFD04460028DFD185
S31508006D3811A8FFF7F5F804460028D8D00428D7D1B3
S31508006D48E1E70246294606A8FEF7F8FE04460028A3
S31508006D58E0D0CDE70624CBE7221400202DE9F3413D
S31508006D6806469046054600244F1EBC4212DA01AB79
S31508006D78012269464046FFF7F5FC019B012B09D11C
S31508006D889DF800300D2BF0D00A2B05F8013B04F1CD
S31508006D980104EAD100239C4214BF304618462B70DA
S31508006DA802B0BDE8F08110B5002394B0CDE90233EE
S31508006DB80191441E14F8011F31B9029A002A07DA0C
S31508006DC84FF0FF3014B010BD01A8FFF736FEF1E703
S31508006DD86B4604A90198FFF76BFD0028F0D1029AC3
S31508006DE8009B9A42ECD10398ECE700007F2810B57F
S31508006DF806D931B1FF2812D880380A4B33F8100063
S31508006E0810BD084A32F8114084428BB203D00131CA
S31508006E188029F7D10B4603F18000C0B2F0E70020BD
S31508006E28EEE700BF9E77000870B51E4B1E4AB0F500
S31508006E38805F28BF1346191D31F8043C0A46A3B1DA
S31508006E48984212D331F8024C250AE4B2E618B04241
S31508006E5821DA082D09D8DFE805F005090F111315F9
S31508006E6817191B00C01A31F8100070BDC31A03F0B1
S31508006E780103C01A80B2F8E71038FBE72038F9E7AB
S31508006E883038F7E71A38F5E70830F3E75038F1E706
S31508006E98A0F5E350EEE70431002DCDD102EB44030B
S31508006EA8C9E700BF9E780008907A00082023038067
S31508006EB800487047480000200A23038000487047A6
S31508006EC86800002008B590F89C32032B01D1FDF71D
S31508006ED8ADFC002008BD08B5FDF7A8FC002008BDD4
S31508006EE808B50846FDF7E0FC002008BD10B5812165
S31508006EF8044600F081F90121204600F07DF90020BA
S31508006F0810BD000010B5402304460222812100F076
S31508006F1863F9402302220121204600F05DF9402347
S31508006F28034A0121204600F0C1F9002010BD00BF20
S31508006F387C1A002010B50A7812F0600F044612D1A0
S31508006F484A780A2A14D00B2A15D0062A0BD14A8859
S31508006F58120A212A09D1CA880B49172A28BF1722D3
S31508006F682046FCF7C1FF002010BD08491722F7E79D
S31508006F7801220749F5E78B7813B9054A1360F2E742
S31508006F88FCF78BFFEFE700BF5A00002051000020EE
S31508006F9824160020004870477C1A002012230B800C
S31508006FA8004870479000002004230B80004870476B
S31508006FB8A400002010B5044C04480A462146FCF7EC
S31508006FC877FF204610BD00BFBC1A00206A7B000860
S31508006FD810B5044C04480A462146FCF769FF2046C2
S31508006FE810BD00BFBC1A0020777B000810B5044CFA
S31508006FF804480A462146FCF75BFF204610BD00BF39
S31508007008BC1A00208A7B000810B5044C04480A46B6
S315080070182146FCF74DFF204610BD00BFBC1A0020CC
S315080070284C7B000810B5044C04480A462146FCF770
S315080070383FFF204610BD00BFBC1A0020547B00083D
S3150800704800F57171D0F80404FCF701BC1C2303FB96
S315080070580103D0F80404D3F80822FCF728BC1C233B
S3150800706803FB0103D0F804049A6CFCF753BCD0F868
S315080070780404FCF7DBBC10B5C1680446003118BF28
S315080070880121D0F80404FCF7BBFCD4F80404BDE8D5
S315080070981040FCF78DBC000010B50446D0F804046F
S315080070A8FCF7B1FC2268D2F8003E43F00103C2F8A7
S315080070B8003E236A23B1044A136943F006031361A1
S315080070C8BDE81040F9F742BA00ED00E010B50446ED
S315080070D8F9F73DFAD4F80404BDE81040FCF79CBC5F
S315080070E8D0F80404FCF7B0BCD0F80404FCF7AABC32
S315080070F810B504460120F9F7FBF9D4F80404BDE8ED
S315080071081040FCF7A3BC10B504460020F9F7F0F9BF
S31508007118D4F80404BDE81040FCF79ABC08B5027810
S3150800712852BB164B0421C3F80404C0F8C4324FF006
S31508007138A040C3E900010221C3E903129961184670
S315080071480121C3E907125A62C3E90B22FAF7CAFAF8
S3150800715820B14FF48D710A48FDF7D6FB8021074800
S31508007168FAF7E8FF402200210448FAF7C3FF80220D
S3150800717801210248FAF7BEFF002008BD281600209C
S315080071889B7B000808B5D0F8C402FAF732FB032837
S3150800719896BF024B0320185C08BD00BF977B000802
S315080071A808B5D0F8C402FAF739FB032896BF024B8C
S315080071B80320185C08BD00BF977B000808B5D0F8FF
S315080071C8C402FAF74AFB032896BF024B0320185C49
S315080071D808BD00BF977B000810B51C46D0F8C40246
S315080071E813462246FAF763FE032896BF014B032087
S315080071F8185C10BD977B000808B5D0F8C402FAF7E2
S315080072088EFE032896BF024B0320185C08BD00BFF4
S31508007218977B000808B5D0F8C402FAF7FBFE0328DE
S3150800722896BF024B0320185C08BD00BF977B000871
S3150800723808B5D0F8C402FAF727FF032896BF024B09
S315080072480320185C08BD00BF977B000811F0800F63
S31508007258D0F8C4324FF01C021BBF01F07F0102FBB5
S31508007268013102FB013191F83E0008BF91F8FE0191
S315080072787047000008B5D0F8C402FAF704FE0328D8
S3150800728896BF024B0320185C08BD00BF977B000811
S3150800729808B5D0F8C402FAF79DFE032896BF024B34
S315080072A80320185C08BD00BF977B000808B5D0F80E
S315080072B8C402FAF763FE032896BF024B0320185C3C
S315080072C808BD00BF977B0008D0F8C402FAF77ABE53
S315080072D870B50D4E0D4CA41BA4100025A54209D166
S315080072E80B4E0C4C00F04EF8A41BA4100025A54222
S315080072F805D170BD56F8253098470135EEE756F89A
S31508007308253098470135F2E7CC7C0008CC7C000884
S31508007318CC7C0008D07C0008044B054A1B681B6A0D
S31508007328002B08BF1346D3F8EC007047A8000020C6
S315080073380C01002082B001B901A942B14BB11378FA
S315080073480B601278101C18BF012002B0704710464F
S31508007358FBE76FF00100F8E702440346934200D1C1
S31508007368704703F8011BF9E749B1FF2A85BF8A2345
S3150800737803600A704FF0FF3098BF0120704708462F
S3150800738870470000F8B500BFF8BC08BC9E467047B1
S31108007398F8B500BFF8BC08BC9E4670475C
S315080073A42F626F6F746C6F672E747874002F646520
S315080073B46D6F70726F675F6F6C696D65785F7374F4
S315080073C46D3332703430352E7372656300000000F5
S315080073D40000000000010203040607080900000073
S315080073E40001020304433A2F576F726B2F736F66BB
S315080073F474776172652F4F70656E424C542F5461D1
S31508007404726765742F536F757263652F41524D43C6
S315080074144D345F53544D333246342F63616E2E63B5
S315080074240005020602060307030803090309040AFA
S31508007434040B040C040C050D050E050F050F0610A8
S31508007444061007100800000000800008004000002D
S315080074540200000000C0000800400000030000000D
S3150800746400000108000001000400000000000208F2
S3150800747400000200050000000000040800000200E5
S3150800748406000000000006080000020007000000CD
S3150800749400000808000002000800000000000A08AE
S315080074A4000002000900000000000C0800000200A9
S315080074B40A00000000000E08000002000B0000008D
S315080074C4433A2F576F726B2F736F667477617265C1
S315080074D42F4F70656E424C542F5461726765742F32
S315080074E4536F757263652F41524D434D345F535440
S315080074F44D333246342F72733233322E6300433A95
S315080075042F576F726B2F736F6674776172652F4F7F
S3150800751470656E424C542F5461726765742F536FAD
S31508007524757263652F41524D434D345F53544D3341
S315080075343246342F7573622E6300083F00303A00D2
S31508007544433A2F576F726B2F736F66747761726540
S315080075542F4F70656E424C542F5461726765742FB1
S31508007564536F757263652F66696C652E6300466989
S31508007574726D7761726520757064617465207265D1
S3150800758471756573742064657465637465640A0D3E
S31508007594004F70656E696E67206669726D776172F1
S315080075A4652066696C6520666F7220726561646918
S315080075B46E672E2E2E004F4B0A0D0053746172749B
S315080075C4696E67207468652070726F6772616D6D85
S315080075D4696E672073657175656E63650A0D00507B
S315080075E4617273696E67206669726D776172652068
S315080075F466696C6520746F206465746563742065B8
S315080076047261736520626C6F636B732E2E2E004550
S31508007614726173696E6720002062797465732066E7
S31508007624726F6D206D656D6F727920617420307884
S315080076340052656164696E67206C696E65206672BE
S315080076446F6D2066696C652E2E2E4552524F520A6E
S315080076540D00496E76616C696420636865636B73B3
S31508007664756D20666F756E642E2E2E4552524F52D6
S315080076740A0D0050726F6772616D6D696E6720003E
S3150800768420627974657320746F206D656D6F7279E5
S315080076942061742030780057726974696E672070A7
S315080076A4726F6772616D20636865636B73756D2E9F
S315080076B42E2E00436C6F73696E67206669726D7748
S315080076C46172652066696C650A0D004669726D7794
S315080076D4617265207570646174652073756363658A
S315080076E4737366756C6C7920636F6D706C657465FD
S315080076F4640A0D004F70656E424C5400809A4541E9
S315080077048E418F804545454949498E8F9092924FBF
S31508007714994F555559999A9B9C9D9E9F41494F55FA
S31508007724A5A5A6A7A8A9AAABACADAEAFB0B1B2B38E
S31508007734B4B5B6B7B8B9BABBBCBDBEBFC0C1C2C37F
S31508007744C4C5C6C7C8C9CACBCCCDCECFD0D1D2D36F
S31508007754D4D5D6D7D8D9DADBDCDDDEDFE0E1E2E35F
S31508007764E4E5E6E7E8E9EAEBECEDEEEFF0F1F2F34F
S31508007774F4F5F6F7F8F9FAFBFCFDFEFF0103050735
S31508007784090E10121416181C1E222A3A3C3E3F7C77
S315080077947F002B2C3B3D5B5D0000C700FC00E90025
S315080077A4E200E400E000E500E700EA00EB00E80098
S315080077B4EF00EE00EC00C400C500C900E600C600F0
S315080077C4F400F600F200FB00F900FF00D600DC0026
S315080077D4A200A300A500A7209201E100ED00F30092
S315080077E4FA00F100D100AA00BA00BF001023AC00C9
S315080077F4BD00BC00A100AB00BB00912592259325D2
S3150800780402252425612562255625552563255125F6
S3150800781457255D255C255B251025142534252C253F
S315080078241C2500253C255E255F255A2554256925F2
S315080078346625602550256C256725682564256525F4
S3150800784459255825522553256B256A2518250C25AF
S31508007854882584258C2590258025B103DF0093038C
S31508007864C003A303C303B500C403A6039803A9036B
S31508007874B4031E22C603B50329226122B100652278
S31508007884642220232123F7004822B0001922B700D6
S315080078941A227F20B200A025A00061001A03E00086
S315080078A41703F8000703FF000100780100013001FF
S315080078B432010601390110014A012E017901060136
S315080078C480014D0043028101820182018401840101
S315080078D486018701870189018A018B018B018D0144
S315080078E48E018F0190019101910193019401F60192
S315080078F496019701980198013D029B019C019D01FF
S3150800790420029F01A001A001A201A201A401A401D1
S31508007914A601A701A701A901AA01AB01AC01AC0103
S31508007924AE01AF01AF01B101B201B301B301B501B3
S31508007934B501B701B801B801BA01BB01BC01BC0164
S31508007944BE01F701C001C101C201C301C401C501D9
S31508007954C401C701C801C701CA01CB01CA01CD01C7
S315080079641001DD0101008E01DE011201F30103009D
S31508007974F101F401F401F8012801220212013A0284
S315080079840900652C3B023B023D02662C3F0240027D
S315080079944102410246020A0153024000810186015E
S315080079A4550289018A0158028F015A0290015C0224
S315080079B45D025E025F02930161026202940164023F
S315080079C4650266026702970196016A02622C6C02D6
S315080079D46D026E029C01700271029D0173027402AB
S315080079E49F0176027702780279027A027B027C0288
S315080079F4642C7E027F02A60181028202A901840206
S31508007A04850286028702AE014402B101B20145022B
S31508007A148D028E028F0290029102B7017B03030046
S31508007A24FD03FE03FF03AC030400860388038903EE
S31508007A348A03B1031103C2030200A303A303C40305
S31508007A440803CC0303008C038E038F03D8031801A1
S31508007A54F2030A00F903F303F403F503F603F70341
S31508007A64F703F903FA03FA03300420035004100752
S31508007A74600422018A043601C1040E01CF04010000
S31508007A84C004D00444016105260400007D1D0100DC
S31508007A94632C001E9601A01E5A01001F0806101F1B
S31508007AA40606201F0806301F0806401F0606511F33
S31508007AB40700591F521F5B1F541F5D1F561F5F1F68
S31508007AC4601F0806701F0E00BA1FBB1FC81FC91FF8
S31508007AD4CA1FCB1FDA1FDB1FF81FF91FEA1FEB1F8C
S31508007AE4FA1FFB1F801F0806901F0806A01F08061A
S31508007AF4B01F0400B81FB91FB21FBC1FCC1F01005A
S31508007B04C31FD01F0206E01F0206E51F0100EC1F73
S31508007B14F21F0100FC1F4E210100322170211002C0
S31508007B24842101008321D0241A05302C2F04602CCB
S31508007B340201672C0601752C0201802C6401002DB4
S31508007B44260841FF1A03000044656661756C7400D3
S31508007B5457696E5553422042756C6B20496E74659D
S31508007B647266616365004F70656E424C54205573A6
S31508007B7465720057696E5553422042756C6B2044F2
S31508007B8465766963650030303030303030303035F2
S31508007B94304300000301032E2E2F5553425F4445FC
S31508007BA4564943452F5461726765742F7573626429
S31508007BB45F636F6E662E6300504F5349580000206A
S31508007BC4202020202020202028282828282020207B
S31508007BD4202020202020202020202020202020882B
S31508007BE4101010101010101010101010101010048F
S31508007BF404040404040404040410101010101010DF
S31508007C0441414141414101010101010101010101D2
S31508007C1401010101010101010101101010101010E8
S31508007C2442424242424202020202020202020202A2
S31508007C3402020202020202020202101010102000BE
S31508007C440000000000000000000000000000000022
S31508007C540000000000000000000000000000000012
S31508007C640000000000000000000000000000000002
S31508007C7400000000000000000000000000000000F2
S31508007C8400000000000000000000000000000000E2
S31508007C9400000000000000000000000000000000D2
S31508007CA400000000000000000000000000000000C2
S31508007CB400000000000000000000000000000000B2
S30D08007CC43485FF7F0100000072
S30908007CCCAD010008F0
S30908007CD08901000810
S31508007CD40024F40001000000100000000104000064
S31508007CE40D6F0008F56E00083D6F000800000000DF
S31508007CF400000000DF6E0008E96E0008CD6E00087B
S31508007D04000000000000000000000000B56E000836
S31508007D1400000000C16E000809022000010100C02D
S31508007D24320904000002FF00000007058102400032
S31508007D34FF070501024000FF0A0610010000004083
S31508007D4401000000A56F0008B16F0008BD6F0008A8
S31508007D54D96F0008F56F0008117000082D70000827
S31508007D641201100100000040501DAC600001010220
S31508007D740301000004030904AC000020000000000D
S31508007D8400000000000000000000000000000000E1
S31508007D9400000000000000000000000000000000D1
S31508007DA400000000000000000000000000000000C1
S31508007DB400000000000000000000000000000000B1
S31508007DC400000000000000000000000000000000A1
S31508007DD4000000000000000000000000430000004E
S31508007DE40000000000000000000000000000000081
S31508007DF4000000000000000000000000430000002E
S31508007E040000000000000000000000000000000060
S31508007E14000000000000000000000000430000000D
S31508007E240000000000000000000000000000000040
S31508007E3400000000000000000000000043000000ED
S31508007E440000000000000000000000000000000020
S31508007E5400000000000000000000000043000000CD
S31508007E640000000000000000000000000000000000
S31508007E7400000000000000000000000043000000AD
S31508007E8400000000000000000000000000000000E0
S31508007E94000000000000000000000000430000008D
S31508007EA400000000000000000000000000000000C0
S31508007EB400000000000000000000000071730008C4
S31508007EC43D73000800000000C27B0008B87500086E
S31508007ED4BE750008BE750008BE750008BE750008A4
S31508007EE4BE750008BE750008BE750008BE75000894
S31508007EF4BE750008FFFFFFFFFFFFFFFFFFFFFFFF41
S31508007F04FFFF0000010041534349490000000000F7
S31508007F14000000000000000000000000000000004F
S31508007F2400000000000041534349490000000000D6
S31508007F34000000000000000000000000000000002F
S30D08007F44000000000000000027
S70508000ABD2B
